:100000000CEF00F000001200D8CFFFF5FACFFEF59C
:04001000EDEF19F007
:10001800110EE96E000EEA6E3F0EE16E020EE26E00
:100028004AEC35F0A50EE96E050EEA6EE20EE16EB9
:10003800050EE26E4AEC35F0E80EE96E000EEA6E47
:10004800000EE16E010EE26E840EF66E000EF76E83
:10005800000EF86E42EC35F0A30EE96E050EEA6E5E
:10006800A50EE16E050EE26E040EF66E000EF76E3A
:10007800000EF86E42EC35F041EF1AF02207DB066D
:100088004907FB0645112E1112115711C811A71166
:100098006F11F510D96AD950130DC20EF324E96E09
:1000A800010EF420EA6EFF0EEE6EED6AD92A020EFA
:1000B800D95CD8B01200EFD7B60EE16E010EE26E31
:1000C80000012B6B00EE0CF0E150E926E250EA2229
:1000D800EE50FF0AED10D8A445D000EE0CF0E15028
:1000E800E926E250EA2225C0EEFF26C0EDFFE1CF67
:1000F8002CF0E2CF2DF0000128512711D8B40ED0F2
:100108002CC05BF02DC05CF027C05DF028C05EF00D
:1001180000010A0E5F6F606B68EC34F02CC0E1FFE1
:100128002DC0E2FF00EE0AF0E150E926E250EA2293
:1001380029C0EEFF2AC0EDFF00EE0EF0E150E926DF
:10014800E250EA22EE6AED6A00EE10F0E150E9268C
:10015800E250EA22000EEE6AED6A2BC0E1F50001DA
:100168002B511200130EE126000EE22200012B2B68
:10017800020E2B5DD8B0FF0CA5D7D96E130DC20E99
:10018800F324E96E010EF420EA6EFF0EEE6E000E07
:10019800ED6A12000001276FE1C5E8FF130DB60EE6
:1001A800F324E16E010EF420E26EE1CF28F0E2CFF5
:1001B80029F000EE0EF0E150E926E250EA22EE5076
:1001C800ED10D8A417D000EE12F02851E9262951D5
:1001D800EA22A7C5EFFF00011C0EBF6FC06B00012C
:1001E80000EE12F02851E9262951EA22EF5071EC6D
:1001F80026F000012751E6EC23F028C0E1FF29C0D2
:10020800E2FF00EE0EF0E150E926E250EA22EE2A83
:10021800000EED2200EE0EF0E150E926E250EA224F
:10022800EECFF3FFEDCFF4FF030EF45CD60ED8B497
:10023800F35CD8B001D8010CE1C5E8FF130DB60E88
:10024800F32400012A6F010EF4202B6F00EE0CF04E
:100258002A51E9262B51EA22EECF00F0EDCF01F02A
:1002680000C0DAF001C0DBF0DFEC2CF000C02CF0AD
:1002780001C02DF0000100EE0AF02A51E9262B51A9
:10028800EA22EECF00F0EDCF01F000C0DAF001C0B5
:10029800DBF0DFEC2CF000C02EF001C02FF00001E5
:1002A80000EE0EF02A51E9262B51EA22EECF00F09B
:1002B800EDCF01F0080E0024E8CF30F0000E012049
:1002C800E8CF31F0326B336B0001140EBF6FC06B97
:1002D800000100EE12F02A51E9262B51EA22EF50D4
:1002E80071EC26F02AC0BFF02BC0C0F0110EE8CF89
:1002F800C1F030C0C2F031C0C3F01FEC2CF030C0E8
:10030800DAF031C0DBF0DFEC2CF000C030F001C0D7
:1003180031F000012C0EE06F000EE16F0001080EB5
:10032800E26FE36BFAEC23F0E7EC25F02AC0E1FF7B
:100338002BC0E2FF00EE12F0E150E926E250EA227B
:10034800FF0EEF6E00EE0EF0E150E926E250EA22D1
:10035800000EEE6AED6A1200D96ED9CFE1F5E1C55B
:10036800E8FF130DC60EF324E96E010EF420EA6EC1
:10037800EF5012002D0043EC24F02DC0E9FF2EC0F1
:10038800EAFFEF6EE1C5E8FF130DC60EF324E96E30
:10039800010EF420EA6EEE06000EED5AE1C5E8FF04
:1003A800130DC60EF324E96E010EF420EA6EEE502A
:1003B800ED10D8A4010CA8EC24F0000CE1C5E8FF6E
:1003C800130DC60EF324E96E010EF420EA6EEE500A
:1003D800ED10D8A4A8EC24F0E1C5E8FF130DC60E73
:1003E800F324E96E010EF420EA6E000EEE6AED6A5F
:0803F80012001B000001200EA1
:10040000556F000E566F0001080E576F586B53EC76
:1004100024F020C0DAF021C0DBF0DFEC2CF000C0CB
:1004200020F001C021F022C0DAF023C0DBF0DFECC5
:100430002CF000C022F001C023F024C0DAF025C067
:10044000DBF0DFEC2CF000C024F001C025F026C06A
:10045000DAF027C0DBF0DFEC2CF000C026F001C0A2
:1004600027F00001200E286F000E296F1BC02AF014
:100470001CC02BF017D800011F6F1F29D8A403D070
:10048000A8EC24F0010C00011F51130DC60EF3243B
:10049000E96E010EF420EA6E24C0EEFF25C0EDFFE8
:1004A000010C280000012C69B60ED96E010EDA6E1F
:1004B000F36A10EE02F02851E1262951E22200EE03
:1004C0000CF0D950E926DA50EA22EE52E652E55015
:1004D000ED18E7CFE8FFD8B4EF18D8A43CD010EE61
:1004E00006F02A51E1262B51E22200EE06F0D95007
:1004F000E926DA50EA22EE50E61808E1EE50E61856
:1005000005E1EE50E61802E1EE50E618D8A420D03E
:1005100028C0E9FF29C0EAFF10EE0AF0D950E12611
:10052000DA50E222E652EE52ED50E518EFCFE8FF46
:10053000D8B4E718D8A40CD000EE10F0D950E926B2
:10054000DA50EA22EE50ED10D8A402D0F350120097
:10055000F35000012C6F130ED926000EDA22F32A75
:10056000020EF35C0001D8A0A4D72C29D8B429D05E
:100570002C51130DB60EF324E96E010EF420EA6E31
:10058000E9CF5BF0EACF5CF0E9CF2DF0EACF2EF0B7
:100590002AC05DF02BC05EF000010A0E5F6F606B39
:1005A00068EC34F028C0E9FF29C0EAFF000110EE32
:1005B0000AF02D51E1262E51E222EECFE6FFEDCFDB
:1005C000E5FF00012C5112005E0ED66EF80ED76EBC
:1005D000070ED56ED58EF284F28A1200FEC100F0AD
:1005E000FFC101F01200F2A41200F80ED76E5E0EE9
:1005F000D66E0101FE2B000EFF238978F2941200C3
:100600005458540048544D00474946004347490058
:100610004A504700434C4100574156007465787476
:100620002F706C61696E0000000000000000000087
:10063000746578742F68746D6C0000000000000011
:1006400000000000696D6167652F67696600000042
:100650000000000000000000746578742F68746D5D
:100660006C0000000000000000000000696D616780
:10067000652F6A7065670000000000000000000040
:100680006170706C69636174696F6E2F6A61766105
:100690002D766D00617564696F2F782D77617665B1
:1006A0000000000000000000485454502F312E304C
:1006B00020323030204F4B0D0A436F6E74656E74DC
:1006C0002D747970653A20000D0A0D0A00474554D3
:1006D00000494E4445582E48544D00485454502F1C
:1006E000312E3020323030204F4B0D0A436F6E7464
:1006F000656E742D747970653A2000485454502FFB
:10070000312E3020353033200D0A0D0A53657276B4
:1007100069636520556E617661696C61626C650D17
:100720000A00485454502F312E3020343034204E9B
:100730006F7420666F756E640D0A0D0A4E6F74201B
:10074000666F756E642E0D0A000D0A0D0A003C6876
:10075000746D6C3E3C686561643E3C7469746C65A4
:100760003E5765622053657276657220492F4F208F
:10077000436F6E74726F6C3C2F7469746C653E3C91
:100780002F686561643E3C626F64793E3C63656ED0
:100790007465723E3C666F6E7420666163653D6889
:1007A000656C7665746963613E3C68323E3C753EBB
:1007B0004F757470757420436F6E74726F6C3C2F3C
:1007C000753E3C2F68323E3C464F524D204D4554BD
:1007D000484F443D47455420616374696F6E3D3016
:1007E0003E3C7461626C6520626F726465723D327A
:1007F0003E3C74723E3C74643E3C696E707574207D
:10080000747970653D7375626D6974206E616D6594
:100810003D312076616C75653D44363D2530313E75
:100820003C2F74643E3C74643E3C696E7075742069
:10083000747970653D7375626D6974206E616D6564
:100840003D302076616C75653D44353D2530303E48
:100850003C2F74643E3C2F74723E3C2F7461626C7A
:10086000653E3C2F666F726D3E3C2F626F64793E31
:100870003C2F68746D6C3E04FFFFFF3C48544D4CA8
:100880003E3C484541443E3C5449544C453E4D69EC
:1008900063726F63686970205443502F495020532E
:1008A0007461636B2044656D6F3C2F5449544C4513
:1008B0003E3C2F484541443E3C4652414D45534500
:1008C0005420726F77733D223130302C3330222028
:1008D000626F726465723D303E20203C4652414D4D
:1008E00045206E616D653D22746F70222009737220
:1008F000633D226D61696E2E68746D22206D617298
:1009000067696E6865696768743D35206D617267F7
:10091000696E77696474683D353E093C4652414DC5
:100920004553455420636F6C733D2238302C38306A
:100930002220626F726465723D303E202009093CBE
:100940004652414D45206E616D653D226C65667471
:10095000222020207372633D225374617475732EBC
:1009600063676922206D617267696E68656967688F
:10097000743D32206D617267696E77696474683D99
:10098000323E202009093C4652414D45206E616DA2
:10099000653D227269676874222020207372633D6E
:1009A00022436F6D6D616E64732E63676922206DE3
:1009B000617267696E6865696768743D32206D6150
:1009C0007267696E77696474683D323E093C2F46F0
:1009D00052414D455345543E3C2F4652414D45539F
:1009E00045543E3C2F48544D4C3E04FFFFFF3C48CD
:1009F000544D4C3E3C484541443E3C2F48454144C3
:100A00003E3C424F44593E3C666F6E7420666163C3
:100A1000653D68656C7665746963613E3C63656ECF
:100A20007465723E3C423E3C553E3C464F4E54201F
:100A300053495A453D3720434F4C4F523D222330B6
:100A40003030306666223E3C503E4D6963726F63C3
:100A5000686970205443502F495020537461636B70
:100A60003C2F503E3C2F423E3C2F553E3C2F464FA4
:100A70004E543E3C2F63656E7465723E54686973D4
:100A800020697320612073616D706C6520706167EF
:100A90006520696E74656E64656420746F2064659A
:100AA0006D6F6E737472617465204D6963726F63EC
:100AB000686970205443502F495020537461636B10
:100AC000206361706162696C69746965732E546832
:100AD000697320706167652069732073657276653C
:100AE00064206279204854545020536572766572B0
:100AF0002C2072756E6E696E67206F6E204D696373
:100B0000726F63686970205049433138206D6963A2
:100B1000726F636F6E74726F6C6C65722C75746932
:100B20006C697A696E67204D6963726F636869707A
:100B3000205443502F495020537461636B2E3C70F6
:100B40003E4D6963726F6368697020537461636BB3
:100B5000206F666665727320666F6C6C6F77696E66
:100B6000672066656174757265733A3C2F703E3C10
:100B7000756C3E3C6C693E506F727461626C6520AE
:100B80006163726F7373204D6963726F636869701C
:100B90002050494331382066616D696C79206F6659
:100BA000206D6963726F636F6E74726F6C6C6572C7
:100BB000733C2F6C693E3C6C693E436F6F7065728D
:100BC0006174697665206D756C74697461736B69A5
:100BD0006E67205443502F495020737461636B3CFF
:100BE0002F6C693E3C6C693E5573652069742061C9
:100BF000732070617274206F6620485454502053E3
:100C00006572766572206F7220637573746F6D20E4
:100C10005443502F495020626173656420617070A5
:100C20006C69636174696F6E3C2F6C693E3C6C69E2
:100C30003E4D756C7469706C652054435020736F21
:100C4000636B657420737570706F72743C2F6C6980
:100C50003E3C6C693E485454502053657276657230
:100C60002077697468206D756C7469706C65206399
:100C70006F6E6E656374696F6E7320737570706FDD
:100C800072743C2F6C693E3C6C693E5061676573C1
:100C9000206D61792062652073746F7265642069CC
:100CA0006E20696E7465726E616C2070726F67720F
:100CB000616D206D656D6F7279206F72206578743B
:100CC00065726E616C206461746120454550524FBD
:100CD0004D3C2F6C693E3C6C693E537570706F7271
:100CE0007420666F722048544D4C20666F726D738D
:100CF0003C2F6C693E3C6C693E50432062617365D9
:100D0000642070726F6772616D20746F20636F6E04
:100D100076657274207765622070616765732069FB
:100D20006E746F204D6963726F63686970204669E5
:100D30006C652053797374656D20284D5046532996
:100D40003C2F6C693E3C6C693E4D6F64756C617202
:100D50002064657369676E20746F20656173696CC8
:100D60007920616464206E657720636F6D706F6EAB
:100D7000656E74733C2F6C693E3C2F756C3E3C2F46
:100D8000424F44593E3C2F48544D4C3E04FFFFFF18
:100D90003C68746D6C3E3C6D657461206874747061
:100DA0002D65717569763D2272656672657368227C
:100DB00020636F6E74656E743D2233223E3C68651D
:100DC00061643E3C7469746C653E5765622053658E
:100DD00072766572205374617475733C2F746974F4
:100DE0006C653E3C2F686561643E3C626F64793E91
:100DF0003C63656E7465723E3C666F6E742066611E
:100E000063653D68656C7665746963613E3C753EFB
:100E10003C68323E53797374656D20537461747508
:100E2000733C2F68323E3C2F753E3C7461626C65AA
:100E300020626F726465723D323E3C74723E3C7457
:100E4000643E53333D2530343C2F74643E3C74641F
:100E50003E44363D2530313C2F74643E3C74643E44
:100E600044353D2530303C2F74643E3C74643E4133
:100E70004E303D2530323C2F74643E3C74643E411C
:100E80004E313D2530333C2F74643E3C2F74723E0E
:100E90003C2F7461626C653E3C62723E3C2F626F17
:100EA00064793E3C2F68746D6C3E04FFFFFF004E7A
:100EB00007434F4D4D414E44532E434749007B0855
:100EC000494E4445582E48544D20202000EE094DEF
:100ED00041494E2E48544D2020202000900D53545F
:100EE000415455532E434749202004FFFF454E44AB
:100EF000204F462046415420204D434850537461B2
:100F0000636B2076322E313100444843502F476CBA
:100F100065616E696E672E2E2E00426F61726420CD
:100F200053657475702E2E2E002020202020202046
:100F300020202020202020202000434F4D4D414ED6
:100F400044532E43474900494E4445582E48544D7A
:100F5000000D0A0D0A0D4D434850537461636B2018
:100F600044656D6F204170706C69636174696F6E68
:100F70002076312E3020284D6963726F6368697066
:100F8000205443502F495020537461636B20322EFC
:100F900030290D0A0D0A09313A204368616E6765F0
:100FA00020426F6172642073657269616C206E7596
:100FB0006D6265722E0D0A09323A204368616E67D0
:100FC000652064656661756C7420495020616464B5
:100FD000726573732E0D0A09333A204368616E6798
:100FE000652064656661756C7420676174657761FE
:100FF0007920616464726573732E0D0A09343A2096
:101000004368616E67652064656661756C74207302
:1010100075626E6574206D61736B2E0D0A09353A29
:1010200020456E61626C652044484350202620496B
:101030005020476C65616E696E672E0D0A09363A5D
:101040002044697361626C65204448435020262027
:10105000495020476C65616E696E672E0D0A09372D
:101060003A20446F776E6C6F6164204D5046532078
:10107000696D6167652E0D0A09383A2053617665FE
:10108000202620517569742E0D0A0D0A456E74656F
:10109000722061206D656E752063686F69636520DD
:1010A00028312D38293A20000D0A496E76616C6985
:1010B0006420696E70757420726563656976656415
:1010C000202D20496E7075742069676E6F7265649B
:1010D0002E0D0A507265737320616E79206B6579ED
:1010E00020746F20636F6E74696E75652E2E2E0DE1
:1010F0000A002575000D0A4E6F772072756E6E69B5
:101100006E67206170706C69636174696F6E2E2EFA
:101110002E000D0A44656661756C74204761746524
:1011200077617920416464726573732028000D0A29
:1011300044656661756C7420495020416464726531
:1011400073732028000D0A53657269616C204E7517
:101150006D6265722028000D0A44656661756C74C5
:10116000205375626E6574204D61736B2028000DED
:101170000A526561647920746F20646F776E6C6FBA
:101180006164204D50465320696D616765202D20B4
:1011900055736520586D6F64656D2070726F746F44
:1011A000636F6C2E0D0A000D0A4448435020262020
:1011B000495020476C65616E696E67206469736190
:1011C000626C65642E0D0A000D0A444843502026C7
:1011D00020495020476C65616E696E6720656E61BD
:1011E000626C65642E0D0A00D96AD950220D0C0E6E
:1011F000F324E16E010EF420E26EE76A00EE21F0C6
:10120000E150E926E250EA22EF50FE0BEF6E00EECD
:1012100021F0E150E926E250EA22EF50FD0B0209ED
:10122000EF6E00EE21F0E150E926E250EA22EF50A5
:10123000FB0B0409EF6E00EE21F0E150E926E250CD
:10124000EA22EF50EF0BEF6E00EE21F0E150E926BD
:10125000E250EA22EF50F70BEF6E00EE0FF0E15094
:10126000E926E250EA22FF0EEF6E00EE1FF0E15099
:10127000E926E250EA22580EEE6E020EED6ED92AF1
:10128000050ED95CD8A0B1D70101006B040E016F27
:101290000101046B056B066B076B12001600D96A1F
:1012A000D950220D0C0EF324E16E010EF420E26EF3
:1012B000E750D8A447D0010EE76E00EE0BF0E150E6
:1012C000E926E250EA2216C0EEFF17C0EDFF00EE5D
:1012D0000DF0E150E926E250EA22EE6AED6A00EEF6
:1012E00007F0E150E926E250EA22EE6AEE6AEE6A81
:1012F000ED6AED52ED5200EE21F0E150E926E250A8
:10130000EA22EF50FE0B0109EF6E00EE21F0E150F2
:10131000E926E250EA22EF50F70BEF6E00EE0FF0F5
:10132000E150E926E250EA22FF0EEF6E00EE21F0D6
:10133000E150E926E250EA22EF50FD0B0209EF6E80
:10134000D9501200D92A050ED95CD8B0FE0CA8D706
:10135000D96E220D0C0EF324E96E010EF420EA6E14
:10136000EF50040A000ED8B4010E1200D96E220DFF
:101370000C0EF324E16E010EF420E26ED950000150
:101380007B6FE1CF7CF0E2CF7DF0E750040AD8B468
:1013900006D07CC07EF07DC07FF0A1EF10F0000190
:1013A0007B51F2D97CC0E1FF7DC0E2FF010EE12458
:1013B000E8CF87F0000EE220E8CF88F000EE0BF0D7
:1013C000E150E926E250EA22EECF00F0EDCF01F045
:1013D00000C089F001C08AF000EE0DF0E150E9266E
:1013E000E250EA22EECF00F0EDCF01F000C08BF02A
:1013F00001C08CF000EE14F0E150E926E250EA2240
:10140000EECF8DF0EECF8EF0EECF8FF0EDCF90F0EF
:10141000ED52ED5200EE18F0E150E926E250EA22DA
:10142000EECF91F0EECF92F0EECF93F0EDCF94F0BF
:10143000ED52ED52110EE8CF95F0FF0EE8CF96F089
:101440000001976B986B85DB7CC0E1FF7DC0E2FFFC
:1014500000EE14F0E150E926E250EA22EE2A000EF6
:10146000EE22EE22ED22ED52ED52050EE76E120055
:10147000D96E220D0C0EF324E16E010EF420E26E03
:1014800000EE0FF0E150E926E250EA22EF50006E44
:101490000028D8B4000C00EE21F0E150E926E2501B
:1014A000EA22EF50006E00A2000C010EE124E8CF0A
:1014B00087F0000EE220E8CF88F000EE0BF0E1505C
:1014C000E926E250EA22EECF00F0EDCF01F000C0B5
:1014D00089F001C08AF000EE0DF0E150E926E250FB
:1014E000EA22EECF00F0EDCF01F000C08BF001C09A
:1014F0008CF000EE14F0E150E926E250EA22EECF43
:101500008DF0EECF8EF0EECF8FF0EDCF90F0ED526C
:10151000ED5200EE18F0E150E926E250EA22EECF5B
:1015200091F0EECF92F0EECF93F0EDCF94F0ED523C
:10153000ED52100EE8CF95F000EE0FF0E150E926E5
:10154000E250EA22EF50E8CF96F000EE10F0E150C2
:10155000E926E250EA22EECF00F0EDCF01F000C024
:1015600097F001C098F0E1CF85F0E2CF86F0F1DA94
:1015700085C0E1FF86C0E2FF00EE14F0E150E926ED
:10158000E250EA22EECF08F1EECF09F1EECF0AF1F8
:10159000EDCF0BF1ED52ED5200EE10F0E150E926E7
:1015A000E250EA22EECF00F0EDCF01F000C002F1F0
:1015B00001C003F100EE10F0E150E926E250EA220A
:1015C000EECF00F0EDCF01F000EE14F0E150E9268F
:1015D000E250EA220050EE260150EE22000EEE22EA
:1015E000ED22ED52ED5200EE14F0E150E926E2500A
:1015F000EA22EECF08F1EECF09F1EECF0AF1EDCFFE
:101600000BF1ED52ED5200EE21F0E150E926E250EF
:10161000EA22EF50FD0BEF6E00EE21F0E150E926DB
:10162000E250EA22EF50EF0BEF6E000100EE0FF0F8
:101630008551E9268651EA22EF5095EC24F085C0C9
:10164000E1FF86C0E2FF00EE0FF0E150E926E25034
:10165000EA22FF0EEF6E00EE21F0E150E926E250A3
:10166000EA22EF50FD0B0209EF6E010CD96E220D3C
:101670001B0EF324E96E010EF420EA6EEF50006EAB
:101680000028D8B4DFEF23F0D950220D2D0EF3241B
:10169000E96E010EF420EA6EEF30010B12007F00BC
:1016A000D96E220D0C0EF3240001836F010EF4207D
:1016B000846FD950806F00EE0FF08351E92684517A
:1016C000EA22EF50006E0028D8A428D000EE0FF0D8
:1016D0008351E9268451EA22A7C5EFFF00EE0FF0FF
:1016E0008351E9268451EA22EF5084EC24F0000172
:1016F00000EE10F08351E9268451EA22EE6AED6A89
:101700000001280EBF6FC06B000100EE0FF0835187
:10171000E9268451EA22EF5071EC26F0000100EE38
:1017200010F08351E9268451EA22EECF81F0EDCF0B
:1017300082F0030E825DCA0ED8B4815DD8B0000C71
:1017400000EE21F08351E9268451EA22EF50EF0B9D
:101750001009EF6E7F51E6EC23F00001814B822BE4
:1017600000EE10F08351E9268451EA2281C0EEFF99
:1017700082C0EDFF030E825DCA0ED8B4815DD8A091
:10178000010C805175DE010CD96E220D0C0EF32474
:10179000E16E010EF420E26EE1CF7EF0E2CF7FF049
:1017A00000EE21F0E150E926E250EA22EF50006E0F
:1017B00000A6000CA8EC24F0000100EE21F07E5100
:1017C000E9267F51EA22EF50F70BEF6E010C15006E
:1017D000D96E220D0C0EF324E16E010EF420E26EA0
:1017E00000EE21F0E150E926E250EA22EF50006ECF
:1017F00000A633D0E1CF15F0E2CF16F000EE21F0D5
:10180000E150E926E250EA22EF50006E00A410D029
:101810000001280E7F6F806B62EC26F0000100EE65
:1018200021F01551E9261651EA22EF50FB0BEF6E1D
:10183000000100EE21F01551E9261651EA22EF5081
:10184000EF0B1009EF6E15C055F016C056F017C01B
:1018500057F018C058F053EF24F0006A016A1200E4
:101860007B00D96E220D0C0EF324E16E010EF420E4
:10187000E26E00EE21F0E150E926E250EA22EF505C
:10188000006E00A6000CE1CF7DF0E2CF7EF000EE0E
:1018900021F0E150E926E250EA22EF50006E00A468
:1018A00010D00001280E7F6F806B62EC26F00001E3
:1018B00000EE21F07D51E9267E51EA22EF50FB0B2C
:1018C000EF6E000100EE12F07D51E9267E51EA2212
:1018D000EE50ED10D8A40DD0A8EC24F0000100EEDD
:1018E00021F07D51E9267E51EA22EF50F70BEF6E91
:1018F000000C000100EE12F07D51E9267E51EA2233
:10190000EE06000EED5A43EC24F07BC0E9FF7CC0EC
:10191000EAFFEF6E010CD96E220D2D0EF324E96E55
:10192000010EF420EA6EEF30006E00320030010B41
:10193000120012001B0000012E0E556F000E566F94
:101940000001140E576F586B53EC24F000012E0E5B
:10195000BF6F000EC06F2EDB000100EE06F01B51C2
:10196000E9261C51EA22EECF22F0EECF23F0EECF93
:1019700024F0EDCF25F0ED52ED5200C226F001C269
:1019800027F002C228F003C229F02A6B060EE8CF26
:101990002BF01DC02CF01EC02DF02CC0DAF02DC095
:1019A000DBF0DFEC2CF000C02CF001C02DF00001CA
:1019B000220ED86F000ED96F00010C0EDA6FDB6BB0
:1019C00046EC2DF0001C026E011C036E02C020F0DC
:1019D00003C021F00001240E7F6F806B62EC26F0C3
:1019E00000EE20F0EF50E6EC23F000EE21F0EF5097
:1019F000E6EC23F00001140E7F6F806B62EC26F0A2
:101A00001DC0BFF01EC0C0F0B6D900C020F001C09C
:101A100021F000EE3EF00001EE522151ED18D8B455
:101A200020C0E8FFEF18D8B403D0A8EC24F0010CD4
:101A300000013A390F0B006ED8900036D890003470
:101A4000EC0FD96E1D5D006E1E51D8A01E05016EF3
:101A5000EC0E00241D6FFF0E01201E6F3A390F0B94
:101A6000006E016AD89000360136D89000360136F3
:101A7000140E0024E8CF7FF0000E0120E8CF80F0A4
:101A800062EC26F000012E0E426F000E436F1BC069
:101A900044F01CC045F0BDD900011F6FFE0E1F5D54
:101AA000D8B011D01BC042F01CC043F000012E0E74
:101AB000446F000E456F1DC046F01EC047F0000188
:101AC0001F51C3DB010CA8EC24F000011F29D8A48E
:101AD000010C1DC000F01EC001F0026A036A005034
:101AE00036270150372302503823035039233BB3A4
:101AF00002D03BA106D00001362B000E372338233D
:101B000039231BC087F01CC088F030C089F031C079
:101B10008AF02EC08BF02FC08CF036C08DF037C00D
:101B20008EF038C08FF039C090F032C091F033C0E1
:101B300092F034C093F035C094F0040EE8CF95F0E5
:101B4000FF0EE8CF96F00001976B986B02D8010C5E
:101B50008700DFEC23F00009D8B4FBD789C0ABF0D5
:101B60008AC0ACF08BC0ADF08CC0AEF08DC0AFF0D1
:101B70008EC0B0F08FC0B1F090C0B2F091C0B3F0A1
:101B800092C0B4F093C0B5F094C0B6F00001B85163
:101B90003F0BB86FB751F00BB76F95C0B8F0BCEC06
:101BA00024F000C0B9F001C0BAF00001040EBA5D23
:101BB000000ED8B4B95D000ED8A004D0B96B040EE5
:101BC000BA6F0FD0BA5D370ED8B4B95DD8A006D0C1
:101BD0000001CA0EB927FF0EBA2303D00001B96B6A
:101BE000BA6B0001BB6BBC6BBD6BBE6B0001AB0E77
:101BF000BF6F000EC06FDED9140E00019727000ED4
:101C0000982395A311D0040E9727000E9823020E57
:101C1000E8CF9BF0040EE8CF9CF0E8CF9DF09E6BE0
:101C2000B7510F0B600904D00001B7510F0B5009D9
:101C3000B76F00C29FF001C2A0F002C2A1F003C2C0
:101C4000A2F0000100EE06F08751E9268851EA2251
:101C5000EECFA3F0EECFA4F0EECFA5F0EDCFA6F03F
:101C6000ED52ED52A76B060EE8CFA8F097C0A9F091
:101C700098C0AAF0A9C0DAF0AAC0DBF0DFEC2CF023
:101C800000C0A9F001C0AAF000019F0ED86F000E9D
:101C9000D96F00010C0EDA6FDB6B46EC2DF0001CE7
:101CA000026E011C036E02C0BBF003C0BCF000EE6C
:101CB000BBF0EECF99F0EDCF9AF000019629D8B4A1
:101CC000A7C596F00001140EBF6FC06B00019651BE
:101CD00071EC26F087C0BFF088C0C0F0060EE8CFD8
:101CE000C1F097C0C2F098C0C3F01FEC2CF0000107
:101CF000AB0EE06F000EE16F0001140EE26FE36BBC
:101D0000FAEC23F095A30BD000019B0EE06F000EC0
:101D1000E16F0001040EE26FE36BFAEC23F00001C7
:101D2000140EBF6FC06B0001965171EC26F097C086
:101D3000BFF098C0C0F01FD800C099F001C09AF061
:101D40000001240EBF6FC06B0001965171EC26F0AC
:101D500000EE9AF0EF50E6EC23F000EE99F0EF5031
:101D6000E6EC23F00001BF6BC06B0001965171ECF3
:101D700026F0E7EF25F00001C16BC12BC36BC46BEC
:101D80000001C051016EBF51006EBF07D8A0C0074F
:101D90000110D8B42CD043EC24F00001C26FC15123
:101DA000D8A40FD0C251C325E8CFC3F0C251C3C0DD
:101DB00000F0005CD8B014D0C43F12D00001C32B97
:101DC0000FD00001C251C425E8CFC4F0C251C4C035
:101DD00000F0005CD8B004D0C33F02D00001C42B97
:101DE0000001C151000ED8B4010EC16FC9D700EE79
:101DF000C4F0EF50FF0AE8CFC4F000EEC3F0EF509C
:101E0000FF0AE8CFC3F0C3C000F0C4C001F0120065
:101E100042000001FE0E466F016A0150220D0C0EB9
:101E2000F324D96E010EF420DA6EDF50D8B44ED010
:101E3000000110EE02F04251E1264351E22200EE91
:101E40000BF0D950E926DA50EA22EE52E652E5507C
:101E5000ED18E7CFE8FFD8B4EF18D8A437D0DF509B
:101E6000006E0004D8A402D00150466F42C0E9FFC2
:101E700043C0EAFF10EE0DF0D950E126DA50E2221D
:101E8000E652EE52ED50E518EFCFE8FFD8B4E71870
:101E9000D8A41CD0000110EE06F04451E1264551B3
:101EA000E22200EE07F0D950E926DA50EA22EE509D
:101EB000E61808E1EE50E61805E1EE50E61802E1FA
:101EC000EE50E618D8A402D001501200012A050EE7
:101ED000015CD8A0A2D700014651220D0C0EF324BC
:101EE000E16E010EF420E26E4651FE0AD8B45BD0DA
:101EF000E750006E0004D8A456D0010EE124E8CFCC
:101F00005BF0000EE220E8CF5CF0E1CF47F0E2CFDB
:101F100048F044C05DF045C05EF000010A0E5F6FFE
:101F2000606B68EC34F047C0D9FF48C0DAFF0001AD
:101F300010EE02F04251E1264351E22200EE0BF096
:101F4000D950E926DA50EA22E6CFEEFFE5CFEDFFE1
:101F500042C0E9FF43C0EAFF10EE0DF0D950E12680
:101F6000DA50E222EECFE6FFEDCFE5FF00EE21F002
:101F7000D950E926DA50EA22EF50F70BEF6E00EE67
:101F80000FF0D950E926DA50EA22FF0EEF6E00EE8C
:101F900021F0D950E926DA50EA22EF50FD0B020970
:101FA000EF6E4651120000014651FE0AD8B4FF0CF4
:101FB000FE0CBF00BFC0E9FFC0C0EAFFEECF00F0DB
:101FC000EDCF01F000C0DAF001C0DBF0DFEC2CF067
:101FD000BFC0E9FFC0C0EAFF00C0EEFF01C0EDFFD7
:101FE000000100EE02F0BF51E926C051EA22EECF17
:101FF00000F0EDCF01F000C0DAF001C0DBF0DFEC63
:102000002CF0000100EE02F0BF51E926C051EA2297
:1020100000C0EEFF01C0EDFF00EE04F0BF51E92665
:10202000C051EA22EECFC1F0EECFC2F0EECFC3F046
:10203000EDCFC4F0ED52ED52F4EC2CF0000100EEC7
:1020400004F0BF51E926C051EA2200C0EEFF01C0F2
:10205000EEFF02C0EEFF03C0EEFF00EE08F0BF513E
:10206000E926C051EA22EECFC1F0EECFC2F0EECFAA
:10207000C3F0EDCFC4F0ED52ED52F4EC2CF00001C2
:1020800000EE08F0BF51E926C051EA2200C0EEFF81
:1020900001C0EEFF02C0EEFF03C0EEFF00EE0EF047
:1020A000BF51E926C051EA22EECF00F0EDCF01F09A
:1020B00000C0DAF001C0DBF0DFEC2CF0000100EE34
:1020C0000EF0BF51E926C051EA2200C0EEFF01C068
:1020D000EDFF00EE10F0BF51E926C051EA22EECF2D
:1020E00000F0EDCF01F000C0DAF001C0DBF0DFEC72
:1020F0002CF0000100EE10F0BF51E926C051EA2299
:1021000000C0EEFF01C0EDFF00EE12F0BF51E92666
:10211000C051EA22EECF00F0EDCF01F000C0DAF0BE
:1021200001C0DBF0DFEC2CF0000100EE12F0BF513B
:10213000E926C051EA2200C0EEFF01C0EDFF120007
:102140007E00000100EE0FF07E51E9267F51EA2269
:10215000EF50006E0028D8B41FD000EE0FF07E5173
:10216000E9267F51EA22EF5095EC24F07EC0E1FF92
:102170007FC0E2FF00EE0FF0E150E926E250EA22D4
:10218000FF0EEF6E00EE21F0E150E926E250EA2268
:10219000EF50FD0B0209EF6E7EC0E1FF7FC0E2FF52
:1021A00000EE07F0E150E926E250EA22EE6AEE6A1C
:1021B000EE6AED6AED52ED5200EE0DF0E150E926C7
:1021C000E250EA22000EEE6AED6AE1CF7EF0E2CF45
:1021D0007FF000EE21F0E150E926E250EA22EF50D4
:1021E000006E00B6A8EC24F07EC0E1FF7FC0E2FFE5
:1021F00000EE21F0E150E926E250EA22EF50F70B21
:10220000EF6E00EE1FF0E150E926E250EA22580E90
:10221000EE6E020EED6E00EE21F0E150E926E25086
:10222000EA22EF50EF0BEF6E00EE21F0E150E926CD
:10223000E250EA22EF50006E00A003D0010EE76EDC
:102240001200000EE76A12004200D96E0001486BCE
:10225000D950220D0C0EF324E16E010EF420E26E33
:1022600000EE18F0E150E926E250EA22EECF4BF002
:10227000EECF4CF0EECF4DF0EECF4EF000EE14F07E
:10228000E150E926E250EA22EECF4FF0EECF50F0D7
:10229000EECF51F0EECF52F000EE04F04451E926BB
:1022A0004551EA22EECF57F0EECF58F0EECF59F07D
:1022B000EECF5AF046C000F047C001F0026A036A50
:1022C00000505727015058230250592303505A23D6
:1022D00000EE14F0E150E926E250EA22EECF53F08E
:1022E000EECF54F0EECF55F0EECF56F000EE1CF0EE
:1022F000E150E926E250EA22000EEF6AE1CF49F010
:10230000E2CF4AF0EEEC02F0000100EE1DF0495180
:10231000E9264A51EA2200C0EEFF01C0EDFF49C0A4
:10232000D9FF4AC0DAFF00EE1FF0D950E926DA5093
:10233000EA22580EEE6E020EED6EDF50006E0004C3
:10234000D8A4A6D0A8EC24F049C0D9FF4AC0DAFF2F
:102350000101042B000E05230623072300EE14F0D1
:10236000D950E926DA50EA2204C1EEFF05C1EEFF9A
:1023700006C1EEFF07C1EEFF0001572B000E5823E8
:1023800059235A2300EE18F0D950E926DA50EA22F0
:1023900057C0EEFF58C0EEFF59C0EEFF5AC0EEFF27
:1023A00000EE14F0D950E926DA50EA22EECF53F0CD
:1023B000EECF54F0EECF55F0EECF56F000EE14F025
:1023C000D950E926DA50EA22EE2A000EEE22EE2259
:1023D000ED22ED52ED5244C0E1FF45C0E2FF00EEB8
:1023E0000DF0E150E926E250EA22EF50006E00A223
:1023F00029D0010ED924E8CF5BF0000EDA20E8CF17
:102400005CF042C05DF043C05EF000010A0E5F6FF9
:10241000606B68EC34F049C0D9FF4AC0DAFF44C0B1
:10242000E9FF45C0EAFF10EE0DF0D950E126DA5081
:10243000E222EECFE6FFEDCFE5FF0001120E486F7E
:10244000020E63D20001040E486F57C053F058C00B
:1024500054F059C055F05AC056F000EE04F0E15067
:10246000E926E250EA22EECF57F0EECF58F0EECF59
:1024700059F0EECF5AF000EE07F0D950E926DA50C5
:10248000EA22EE6AEE6AEE6AED6AED52ED5258D239
:1024900044C0E1FF45C0E2FF00EE0DF0E150E92647
:1024A000E250EA22EF50006E00A407D0A8EC24F01E
:1024B00049C07EF04AC07FF044D600EE08F0E150FB
:1024C000E926E250EA220001EE50531908E1EE50ED
:1024D000541905E1EE50551902E1EE505619D8A4F1
:1024E0002DD2DF50020AD8A457D000EE0DF0E150F3
:1024F000E926E250EA22EF50006E00A84AD000EE32
:1025000018F0D950E926DA50EA2257C0EEFF58C039
:10251000EEFF59C0EEFF5AC0EEFF00EE1CF0D9509E
:10252000E926DA50EA22000EEF6AEEEC02F0000132
:1025300000EE1DF04951E9264A51EA2200C0EEFFA3
:1025400001C0EDFF49C0E1FF4AC0E2FF040EE76EA3
:1025500047514611D8B41AD000EE21F0E150E926D7
:10256000E250EA22EF50F70B0809EF6E00EE12F08E
:10257000E150E926E250EA2246C0EEFF47C0EDFFF7
:1025800000EE21F0E150E926E2506DD0A8EC24F0F5
:10259000D7D1A8EC24F0D4D1DF50030AD8A46FD04F
:1025A00000EE0DF0E150E926E250EA22EF50006E15
:1025B00000A262D00001572B000E582359235A2342
:1025C00000EE18F0D950E926DA50EA2257C0EEFFA3
:1025D00058C0EEFF59C0EEFF5AC0EEFF00EE0DF0FE
:1025E000E150E926E250EA22EF50006E00A805D043
:1025F000100E486F040EDF6E18D00001120E486FE7
:10260000020EDF6E532B000E54235523562300EE8B
:1026100014F0D950E926DA50EA2253C0EEFF54C034
:10262000EEFF55C0EEFF56C0EEFF000147514611C8
:10263000D8B41FD000EE21F0D950E926DA50EA22B2
:10264000EF50F70B0809EF6E00EE12F0D950E926B3
:10265000DA50EA2246C0EEFF47C0EDFF00EE21F05F
:10266000D950E926DA50EA22EF50FB0B0409EF6E4D
:1026700067D1A8EC24F064D1A8EC24F061D110EE6D
:1026800018F0D950E126DA50E222000100EE04F001
:102690004451E9264551EA22EE50E61808E1EE5091
:1026A000E61805E1EE50E61802E1EE50E618D8A46F
:1026B000A8EF24F000EE18F0D950E926DA50EA220B
:1026C00057C0EEFF58C0EEFF59C0EEFF5AC0EEFFF4
:1026D000DF50040AD8A4BFD0000100EE0DF0445131
:1026E000E9264551EA22EF50006E00A82AD000EEFC
:1026F0000FF0D950E926DA50EA22EF50006E002898
:10270000D8B41FD000EE0FF04951E9264A51EA2211
:10271000EF5095EC24F049C0D9FF4AC0DAFF00EE33
:102720000FF0D950E926DA50EA22FF0EEF6E00EEE4
:1027300021F0D950E926DA50EA22EF50FD0B0209C8
:10274000EF6E000100EE0DF04451E9264551EA22FA
:10275000EF50006E00A02BD0110E486F00EE14F069
:10276000D950E926DA50EA2224EC35F000C053F0C3
:1027700001C054F002C055F003C056F000EE18F04E
:10278000D950E926DA50EA22EE2A000EEE22EE2295
:10279000ED22ED52ED52EECF57F0EECF58F0EECFE6
:1027A00059F0EDCF5AF0ED52ED520A0EDF6E0001F6
:1027B00047514611D8B44CD000EE21F0D950E9264B
:1027C000DA50EA22EF50006E00B621D000EE21F080
:1027D000D950E926DA50EA22EF50F70B0809EF6EDC
:1027E00000EE12F0D950E926DA50EA2246C0EEFF98
:1027F00047C0EDFF00EE21F0D950E926DA50EA2279
:10280000EF50FB0B0409EF6E100E486F99D00001DA
:10281000486B00EE14F0D950E926DA50EA224FC096
:10282000EEFF50C0EEFF51C0EEFF52C0EEFF00EED3
:1028300018F0D950E926DA50EA224BC0EEFF4CC01E
:10284000EEFF4DC0EEFF4EC0EEFFA8EC24F078D0B6
:10285000A8EC24F075D0DF500A0AD8A413D0A8EC55
:1028600024F0000100EE0DF04451E9264551EA2222
:10287000EF50006E00A864D049C07EF04AC07FF0DF
:1028800060DC5ED0DF50050AD8A441D0A8EC24F06B
:1028900044C0E1FF45C0E2FF00EE0DF0E150E92643
:1028A000E250EA22EF50006E00A04AD00001100E64
:1028B000486F49C0D9FF4AC0DAFF00EE18F0D9507E
:1028C000E926DA50EA22EE2A000EEE22EE22ED226E
:1028D000ED52ED52EECF57F0EECF58F0EECF59F06B
:1028E000EDCF5AF0ED52ED5200EE0DF0E150E92639
:1028F000E250EA22EF50006E00A806D0D9CF7EF059
:10290000DACF7FF01EDC1CD0060EDF6E19D0DF5050
:10291000060AD8A415D0A8EC24F0000100EE0DF0B2
:102920004451E9264551EA22EF50006E00A808D034
:1029300049C07EF04AC07FF004DC02D0A8EC24F04D
:1029400000014851D8B4120042C087F043C088F05B
:1029500044C0E1FF45C0E2FF00EE02F0E150E9268D
:10296000E250EA22EECF00F0EDCF01F000C089F096
:1029700001C08AF0E6CF00F0E5CF01F000C08BF097
:1029800001C08CF053C08DF054C08EF055C08FF054
:1029900056C090F057C091F058C092F059C093F0D3
:1029A0005AC094F048C095F0FF0EE8CF96F00001B1
:1029B000976B986BA9EF0DF00001156B0001500E9D
:1029C000166F176B4FEC09F0006E000115510A0DE0
:1029D000DC0EF324E96E010EF420EA6E00C0EFFF76
:1029E00015510A0DDF0EF324E96E010EF420EA6E94
:1029F000EF6A152B030E155DD8B01200DFD700016A
:102A0000156B0001155107D80001152B030E155D3C
:102A1000D8B01200F6D7D96E0A0DDC0EF3240001EF
:102A20001E6F010EF4201F6F176B172B000117513B
:102A3000D8B41200176B1EC0E9FF1FC0EAFFEF50A9
:102A4000A8EC09F00009000100EE03F0D8A410D2B0
:102A50001E51E9261F51EA22000EEF6A12001EC025
:102A6000E9FF1FC0EAFFEF508BEC0CF000090001FA
:102A7000D8B4DDD7176B172B1A6B1B6B0001000E38
:102A80001B5D500ED8B41A5DD8B01AD01B51016E20
:102A90001A51006E1A4B1B2B2A0FE8CF7BF0000E49
:102AA0000120E8CF7CF01EC0E9FF1FC0EAFFEF5015
:102AB00031EC0CF0006E016A01500010D8A4DED792
:102AC000000100EE2AF01A51E9261B51EA22000EFD
:102AD000EF6A1EC0E9FF1FC0EAFFEF50C4EC0BF025
:102AE000000100EE03F01E51E9261F51EA22020EFA
:102AF000EF6E050E186F00012A0E7B6F000E7C6FC3
:102B00000001200E7D6F000E7E6F0001180E7F6F9A
:102B1000000E806F0001090E1E25E8CF81F0000E27
:102B20001F21E8CF82F0C4DA0001166F0009D8A493
:102B30007DD7020E185DD8A012D00001200E7B6F49
:102B4000000E7C6F18C07DF0D4EC1BF0000100EE8D
:102B500009F01E51E9261F51EA22030EEF6E20C034
:102B60007BF021C07CF0BDEC30F0000100EE01F004
:102B70001E51E9261F51EA2200C0EEFF01C0EDFF01
:102B80001EC0E1FF1FC0E2FF00EE01F0E150E926A8
:102B9000E250EA22EE52ED50FF0AFF0ED8B4EF18D1
:102BA000D8A411D000EE08F0E150E926E250EA2264
:102BB000000EEF6E00EE03F0E150E926E250EA224B
:102BC000020EEF6E33D700EE01F0E150E926E2503D
:102BD000EA22EE50ED10D8A408D000EE08F0E15043
:102BE000E926E250EA22030EE4D700EE03F0E150BA
:102BF000E926E250EA220B0EE4D71EC0E9FF1FC00F
:102C0000EAFFEF5036EC0BF000090001D8B40FD703
:102C100000EE08F01E51E9261F51EA22EF50006E27
:102C2000016AD8900034026E0134036EE80E02246B
:102C3000E96E000E0320EA6EEECF1CF0EDCF1DF022
:102C400000011CC0F6FF1DC0F7FF010E1C27000E7F
:102C50001D23050EF76403D00800F55005D0F6CF0C
:102C6000E9FFF7CFEAFFEF50D96E0009D8B40AD0D8
:102C7000D9CF7FF01EC0E9FF1FC0EAFFEF5050EC34
:102C80000BF0DED71EC0E9FF1FC0EAFFEF5038ECA3
:102C90000AF0C1D01EC0E9FF1FC0EAFFEF5036ECBA
:102CA0000BF000090001D8B4C2D6176B172B196BB3
:102CB0001951006E016A0050A80FF66E0150F76EB0
:102CC000060EF7220800F550E8CF7FF01EC0E9FF9E
:102CD0001FC0EAFFEF5050EC0BF00001192B1F0E44
:102CE000195DD8A0E5D700EE09F01E51E9261F5165
:102CF000EA22EF50140D1C0EF3241C6F060EF42074
:102D00001D6F00011CC0F6FF1DC0F7FF010E1C2740
:102D1000000E1D23050EF76403D00800F55005D002
:102D2000F6CFE9FFF7CFEAFFEF50D96E0009D8B42C
:102D30000AD0D9CF7FF01EC0E9FF1FC0EAFFEF50D5
:102D400050EC0BF0DED70001196B00011951006E39
:102D5000016A0050C80FF66E0150F76E060EF7229A
:102D60000800F550E8CF7FF01EC0E9FF1FC0EAFF62
:102D7000EF5050EC0BF00001192B040E195DD8A098
:102D8000E4D71EC0E1FF1FC0E2FF00EE09F0E150F2
:102D9000E926E250EA22EF50030A00EE07F0D8A439
:102DA00006D0E150E926E250EA22010E05D0E150BA
:102DB000E926E250EA22000EEF6E00EE04F0E15048
:102DC000E926E250EA22030EEF6E00EE03F0E15036
:102DD000E926E250EA22010EF4D61EC0E9FF1FC028
:102DE000EAFFEF508BEC0CF00009D8B407D01EC0FE
:102DF000E9FF1FC0EAFFEF50C4EC0BF01EC07BF0F0
:102E00001FC07CF047D8006E016A01500010D8B492
:102E10000DD657EC31F0000100EE03F01E51E9260B
:102E20001F51EA22090ECDD61EC0E9FF1FC0EAFFDE
:102E3000EF50A8EC09F00009D8B4F8D51EC0E9FF9E
:102E40001FC0EAFFEF5036EC0BF00009D8B4EED506
:102E50001EC0E9FF1FC0EAFFEF50B6EC09F0000109
:102E600000EE03F01E51E9261F51EA220A0EA9D6F0
:102E70001E51E9261F51EA22EF5001E1F0D5010A67
:102E8000ACE0030A01E1B9D60B0ACEE0020A01E187
:102E900001D7CCD5000100EE01F07B51E9267C5131
:102EA000EA22EECF00F0EDCF01F000C0FCF101C04E
:102EB000FDF1B1D000017E51250AD8A408D000EE62
:102EC00004F0E150E926E250EA22050E12D000019A
:102ED0007D6B7D2B93D000017E51250AD8A40BD0A9
:102EE0007D6B7D2B00EE04F0E150E926E250EA22F2
:102EF000030EEF6E83D000EE08F0E150E926E250B9
:102F0000EA227EC000F0D00E00260038F00BEF6EF3
:102F100000EE04F0E150E926E250EA22060EE9D77D
:102F20007EC000F0D00E002600EE08F0E150E92649
:102F3000E250EA220050EF1200EE04F0E150E926E0
:102F4000E250EA22080EEF6E00EE05F0E150E926AD
:102F5000E250EA22EE6AED6A51D0000100EE05F07F
:102F60007B51E9267C51EA22EECF00F0EDCF01F053
:102F700000C07FF001C080F000017E0E816F000E66
:102F8000826F000100EE08F07B51E9267C51EA22B5
:102F9000EF5028EC1CF0000100EE05F07B51E92613
:102FA0007C51EA2200C0EEFF01C0EDFF7D6B7D2B5E
:102FB0007BC0E1FF7CC0E2FF00EE05F0E150E926B6
:102FC000E250EA22EE52ED50FF0AFF0ED8B4EF189D
:102FD000D8A414D087D7FFD700EE04F0E150E9263B
:102FE000E250EA22EF50030A01E164D7060A01E148
:102FF00072D7030A95E00E0AB0E0EDD700017D51CB
:10300000D8B409D07EC07FF07BC0E9FF7CC0EAFF66
:10301000EF5050EC0BF07BC0E9FF7CC0EAFFEF50B3
:1030200036EC0BF000090001D8B436D07D6B00EE11
:1030300004F07B51E9267C51EA22EF50080AD8B40B
:1030400014D06AEC31F000017E6F0101FD51FF0ADE
:10305000FF0ED8B4FC19D8A408D07BC0E9FF7CC00F
:10306000EAFFEF5038EC0AF0010C7BC0E1FF7CC0B6
:10307000E2FF00EE07F0E150E926E250EA22EF50CD
:10308000D8A4AAD77EC07FF07BC0E9FF7CC0EAFF4E
:10309000EF5050EC0BF0BFD700EE01F07B51E9266A
:1030A0007C51EA22FCC1EEFFFDC1EDFF000C7B006C
:1030B0000001846B896B8A6B856B7BC08BF07CC055
:1030C0008CF00001CD0E8D6F060E8E6F0001030E89
:1030D0008F6F906BCFEC33F001500010D8A4020C2E
:1030E0007BC0E1FF7CC0E2FF040EE126000EE2227D
:1030F0000001836B02D0E14AE22AE750200AD8B4EB
:10310000FAD79FD07FC0E9FF80C0EAFFEF500001EF
:10311000855DD8B0A6D087D000018551006E016AC8
:10312000D8900034026E0134036ED9500224E96E47
:10313000DA500320EA6EE1CFEEFFE2CFEDFFE7CFFA
:10314000F3FFF3502F0AD8B428D0F3505C0AD8A468
:1031500076D023D000018551006E016AD8900034EA
:10316000026E0134036ED9500224E96EDA50032056
:10317000EA6EE1CFEEFFE2CFEDFF852B020E846F0A
:10318000E7CFF3FFF3503F0AD8B404D0F350260A38
:10319000D8A406D0000EE76A0001846B842B4FD0C0
:1031A000F3502B0AD8A403D0200EE76E48D0F3507A
:1031B0002E0AD8A410D000018505D8A40CD0E10EA9
:1031C000E96E0F0EEA6EEE2A000EED22EECF89F0C8
:1031D000EDCF8AF034D0F3503D0AD8B4DBD7F350AA
:1031E0002F0AD8B404D0F3505C0AD8A428D0000128
:1031F0008551006E016AD8900034026E0134036E6E
:10320000D9500224006EDA500320016EFE0E002415
:10321000E96EFF0E0120EA6E010EE124EE6E000E53
:10322000E220ED6E0CD07DC0D9FF7EC0DAFF000138
:10323000845101E171D7010A8DE0030AA1E0E14A5E
:10324000E22AE7CFD9FFD950200AD8B40AD0D95002
:10325000D8B407D00D0AD8B404D0D9500A0AD8A4DB
:1032600051D7000EE76A81C0E9FF82C0EAFF070E6E
:10327000EF6E00018A518911D8B433D089C08FF024
:103280008AC090F0CDEC2DF000C089F001C08AF02A
:103290000001000E876F060E886F866B89C08BF069
:1032A0008AC08CF087C08DF088C08EF00001030EBC
:1032B0008F6F906BCFEC33F001500010D8A407D083
:1032C00081C0E9FF82C0EAFF86C0EFFF0AD0040E8A
:1032D00000018727000E8823862B070E865DD8A065
:1032E000DDD700018551D8A42ED07DC0E9FF7EC076
:1032F000EAFFEECF00F0EDCF01F000C08FF001C08B
:1033000090F00001D10E916F060E926F090EE8CF7A
:1033100093F0FEEC2DF07DC0E9FF7EC0EAFFEECF1A
:1033200000F0EDCF01F0090E0024E96E000E01203F
:10333000EA6E000EEF6A81C0E9FF82C0EAFF010E6B
:10334000EF6E0001852B7FC0E9FF80C0EAFF85C0DA
:10335000EFFF000183511200F3EC02F0E2C5F3FF2E
:10336000E3C5F4FFE4C5F5FFE5C5F6FFE6C5F7FFE5
:10337000E7C5F8FFE8C500F0E9C501F0EAC502F0CD
:10338000EBC503F0ECC504F0EDC505F0EEC506F0A5
:10339000EFC507F0F0C508F0F1C509F0F2C50AF075
:1033A000F3C50BF0F4C50CF0F5C50DF0F6C50EF045
:1033B000F7C5DAFFF8C5D9FFF9C5E2FFFAC5E1FFA5
:1033C000FBC5EAFFFCC5E9FFFDC5E8FFFEC5FAFF46
:1033D000FFC5D8FF0FC0E0FF1000E0CF0FF0E8CF2F
:1033E000FDF5E9CFFCF5EACFFBF5E1CFFAF5E2CF49
:1033F000F9F5D9CFF8F5DACFF7F50EC0F6F50DC02F
:10340000F5F50CC0F4F50BC0F3F50AC0F2F509C0F0
:10341000F1F508C0F0F507C0EFF506C0EEF505C000
:10342000EDF504C0ECF503C0EBF502C0EAF501C010
:10343000E9F500C0E8F5F8CFE7F5F7CFE6F5F6CF08
:10344000E5F5F5CFE4F5F4CFE3F5F3CFE2F584D776
:10345000ACA2FED7AD6E12003F003FC0E1FF40C0FE
:10346000E2FFE250016EE150006EE14AE22A00C044
:10347000E9FF01C0EAFFEF50D96ED8B41200E8DFCF
:10348000F0D7F86A4FDAE4EC02F0B3EC30F068DA27
:1034900081BA0BD0C00E04EC32F000011A0E3F6F5F
:1034A0000F0E406F70EC32F0FCDB2FEC2EF0DCECFA
:1034B00014F018C200F000A00BD0C00E04EC32F0E3
:1034C0000001090E3F6F0F0E406F70EC32F006D016
:1034D000010EE8CFCEF5070EE8CFA3F53FEC2EF0B6
:1034E000FFEC14F00DD9CEC500F0DFC5E8FF0018E1
:1034F000D8B4F4D70001000E326F020E336F010E04
:10350000E8CF34F019D8DFC5CEF518C200F000A01E
:10351000E5D7CE0E04EC32F00A0ECEC500F0005C0A
:10352000CEC5E8FFD8B004D0300F90EC32F0D6D73B
:10353000410F90EC32F0D2D700013451C00ED8B414
:103540000AD004EC32F00001290E3F6F0F0E406FDD
:1035500070EC32F0C00E04EC32F00001350E416F19
:10356000000E426F0001F20E436F100E446F32C026
:10357000E9FF33C0EAFFEF50006E016A00C03DF082
:1035800001C03EF03D0EE8CF3FF0000EE8CF40F026
:1035900094EC26F000013451D8B40BD00001350E64
:1035A0003F6F000E406F59EC32F02E0E90EC32F06F
:1035B00008D00001350E3F6F000E406F4EDF2E0E1B
:1035C00047DF0001350E416F000E426F0001F20E21
:1035D000436F100E446F000100EE01F03251E926F6
:1035E0003351EA22EF50006E016A00C03DF001C085
:1035F0003EF03D0EE8CF3FF0000EE8CF40F094ECF7
:1036000026F000013451D8B40BD00001350E3F6FC5
:10361000000E406F59EC32F02E0E90EC32F008D0D4
:103620000001350E3F6F000E406F17DF2E0E10DFCA
:103630000001350E416F000E426F0001F20E436F24
:10364000100E446F000100EE02F03251E9263351B2
:10365000EA22EF50006E016A00C03DF001C03EF06A
:103660003D0EE8CF3FF0000EE8CF40F094EC26F09E
:1036700000013451D8B40BD00001350E3F6F000E5D
:10368000406F59EC32F02E0E90EC32F008D0000171
:10369000350E3F6F000E406FE0DE2E0ED9DE0001CA
:1036A000350E416F000E426F0001F20E436F100E97
:1036B000446F000100EE03F03251E9263351EA2253
:1036C000EF50006E016A00C03DF001C03EF03D0EBB
:1036D000E8CF3FF0000EE8CF40F094EC26F0000178
:1036E0003451D8B407D00001350E3F6F000E406F43
:1036F00059EF32F00001350E3F6F000E406FADD62E
:10370000810EC26E640EE8CF15F000011507152971
:10371000D8A4FBD7C284C2B4FED7C3CF15F0C4CFA0
:1037200016F00001CF0E416F050E426F0001F20E40
:10373000436F100E446F15C017F016C018F0170E27
:10374000E8CF3FF0000EE8CF40F094EC26F0840E76
:10375000C16E890EC26E640EE8CF15F00001150728
:103760001529D8A4FBD7C284C2B4FED7C3CF15F0A5
:10377000C4CF16F00001D70E416F050E426F000155
:10378000F20E436F100E446F15C017F016C018F0FC
:10379000170EE8CF3FF0000EE8CF40F094EC26F093
:1037A0008E0EC16E12007B007BC0E1FF7CC0E2FF89
:1037B000E6CF00F0E5CF01F000C0E9FF01C0EAFF6D
:1037C000EF50D00FD96E3FD000EE02F0E150E92665
:1037D000E250EA22EECF00F0EDCF01F000C0E9FFA9
:1037E00001C0EAFFEF50D00FD96E04D0897606D021
:1037F000897404D0D950FAE0010AFAE0E6CF00F06B
:10380000E5CF01F000C08FF001C090F000013A0E4A
:10381000916F0F0E926F0D0EE8CF93F0FEEC2DF02E
:103820001200E6CF00F0E5CF01F000C08FF001C03C
:1038300090F00001470E916F0F0E926F0A0EE8CFC5
:1038400093F0FEEF2DF0D950BFE0010AE9E0E9D78F
:10385000E16E56D089B603D050D089A44ED0300E38
:103860004DD0000180517F11D8A402D07F6B806BB6
:1038700000017F5105EECFF0E926000EEA22EFCFDE
:10388000DFFF7F5105EECFF0E926000EEA22EF5070
:10389000D8A404D0FF0E006E016E120000017F4B11
:1038A000802B7FC000F080C001F012000001805129
:1038B0007F11D8A402D07F6B806B00017F5105EE91
:1038C000D7F0E926000EEA22EFCFDFFF7F5105EEA9
:1038D000D7F0E926000EEA22EF50D8A404D0FF0E5C
:1038E000006E016E120000017F4B802B7FC000F044
:1038F00080C001F0120081AAB2D7310EDF6E0ED067
:1039000081C0D9FF82C0DAFFE150A4E0010AA5E03E
:10391000030AA7E0010ACAE0070AEDE0FF0E006E05
:10392000016E12008E0EC16E030E926E809A898413
:103930008986F19EC9EC31F0800E04EC32F0000172
:10394000F90E3F6F0E0E406F70EC32F0200EAC6E31
:10395000900EAB6E0F0EAF6ED56AF28EF28C120027
:103960000A0EE8CF00F2E8CF01F2050EE8CF02F22E
:103970000F0EE8CF03F2FF0EE8CF0AF2E8CF0BF20A
:10398000E8CF0CF202010D6B0A0EE8CF0EF2E8CF81
:103990000FF2050EE8CF10F20F0EE8CF11F2020180
:1039A000046B040EE8CF05F2A30EE8CF06F2020185
:1039B000076B0201086B0201096B02EE18F0EF5071
:1039C000FE0B0109EF6E12003200000132C0F6FF5B
:1039D00033C0F7FF010E3227000E3323050EF764C4
:1039E00003D00800F55005D0F6CFE9FFF7CFEAFF86
:1039F000EF50D96E0009D8B412002ADDE6D732C0E4
:103A0000E1FF33C0E2FFD96A9EAAFED7AE50F36E43
:103A10000D0AD8B40DD0F3500A0AD8B409D0D92A67
:103A2000F3CFE6FFE76A000134073429D8A4ECD7C6
:103A3000D9501200320032C0E1FF33C0E2FFE1CFC3
:103A400037F0E2CF38F00001366BE750D96ED8B4CA
:103A500037D02E0AD8A429D0E250016EE150006E72
:103A6000E14AE22A00C0E9FF01C0EAFF000EEF6A66
:103A7000E1CF32F0E2CF33F037C039F038C03AF05E
:103A8000C6EC32F0000136513425E96E000E3521C6
:103A9000EA6E00C0EFFF362B32C0E1FF33C0E2FF19
:103AA000E1CF37F0E2CF38F008D0300ED95CD8A0A3
:103AB000000C3A0ED95CD8B0000CE14AE22AC5D716
:103AC00037C039F038C03AF0C6EC32F00001365158
:103AD0003425E96E000E3521EA6E00C0EFFF365145
:103AE000030A000ED8B4010E12009EAAFED7AE50F3
:103AF000D96E310ED95C390ED8A01200D95CD8B07D
:103B0000390CD9501200E16E0D0EA2DC0A0EA0DCB9
:103B1000E150006E016AD8900034026E0134036EE9
:103B20008E0E0224E96E000E0320EA6EEECF00F046
:103B3000EDCF01F000C032F001C033F046DF9ED07F
:103B400000011C0E416F000E426F0001F20E436F28
:103B5000100E446F02EE12F0EECF30F0EDCF31F0E8
:103B6000300EE8CF3FF0000EE8CF40F094EC26F0A6
:103B700000011C0E3F6F000E406F6FDC290E68DCE9
:103B80003A0E66DC200E64DC00011C0E326F000E63
:103B9000336F140EE8CF34F032DF006E016A01504B
:103BA0000010D8B447D000011C0E396F000E3A6FD8
:103BB000C6EC32F000C012F201C013F213C208F2D8
:103BC00012C209F21200000EE96E020E07D00E0EAC
:103BD000E96E020E03D00A0EE96E020EEA6EE9CF1C
:103BE00032F0EACF33F0E9CF16F0EACF17F0000158
:103BF000346BA2DC290E2CDC3A0E2ADC200E28DCE9
:103C000000011C0E326F000E336F140EE8CF34F03B
:103C1000F6DE00011C0E326F000E336F0001180E2D
:103C2000346F000E356F07DF006E016A015000101F
:103C3000D8A40AD00001A80E326F100E336FC5DE73
:103C40009EAAFED7AE50120016C0E9FF17C0EAFFC9
:103C500018C0EEFF19C0EEFF1AC0EEFF1BC0EEFF4A
:103C6000120002EE18F0EF50FE0B0109EF6E120089
:103C700002EE18F0EF50FE0BEF6E1200E150310A29
:103C800001E15ED7030A9FE0010AA1E0070AA3E071
:103C9000010AE7E0030AECE0010AEFE00F0AEDE0B9
:103CA00012000001510E326F0F0E336F8EDE1DDFDA
:103CB0000001156F390AD8B402D0155124DF000174
:103CC0001551380AD8B41200ECD70F0EFBEF34F0C0
:103CD000040EFBEF34F0F29ED96AD92AD92EFED712
:103CE000F28E1200FDD1E4D1FF0EE8CF1BF0FF0EE3
:103CF000E8CF1CF0FF0EE8CF1DF0FF0EE8CF1EF05E
:103D0000FF0EE8CF1FF0FF0EE8CF20F0FF0EE8CF48
:103D100021F0E8CF22F0E8CF23F0E8CF24F0020131
:103D2000276B286B296B2A6B0001440E256F266BCD
:103D300000011B0E276F000E286F0001430E296F34
:103D40002A6B60EC00F0E8CFE0F5EEEC02F000C08A
:103D500019F201C01AF2010EE8CFA3F5EEEC02F061
:103D600019C202F01AC203F00350015C02E10250D2
:103D7000005CD8A02DD000D0EEEC02F019C2E8FF14
:103D8000005C026E1AC2E8FF0158036E000E035C6D
:103D9000020ED8B4025C000ED8B0010E006E016AAB
:103DA00018D0EEEC02F000C002F001C003F019C21E
:103DB000F6FF1AC2F7FFFF0E006EFF0E016EF650FF
:103DC000005EF750015A025000260350012201D034
:103DD000E8D701500010D8B401D001D003D0020EB2
:103DE000E8CFA3F57CD102012751281129112A110E
:103DF000D8B401D001D004D0040EE8CFA3F50BD085
:103E0000010E3DDBEEEC02F000C019F201C01AF227
:103E1000030EE8CFA3F563D1E0C5E8FFB0EC01F0F5
:103E20000009D8B401D001D00AD065D9020AD8A4BB
:103E300001D001D003D0040EE8CFA3F544D0EEECBE
:103E400002F019C202F01AC203F00350015C02E151
:103E50000250005CD8A02DD000D0EEEC02F019C2C8
:103E6000E8FF005C026E1AC2E8FF0158036E000E04
:103E7000035C0A0ED8B4025C000ED8B0010E006ECE
:103E8000016A18D0EEEC02F000C002F001C003F0AD
:103E900019C2F6FF1AC2F7FFFF0E006EFF0E016E89
:103EA000F650005EF750015A0250002603500122DE
:103EB00001D0E8D701500010D8B401D001D003D010
:103EC000020EE8CFA3F50BD1E0C5E1F5DFEC23F05E
:103ED0000009D8B401D001D00BD0030ED0DAEEEC3B
:103EE00002F000C019F201C01AF2050EE8CFA3F5E6
:103EF000F6D0E0C5E8FFB0EC01F00009D8B401D07D
:103F000001D035D0F8D8050AD8A401D001D02ED0E0
:103F1000E0C5E8FFC1EC00F0EEEC02F000C019F2E1
:103F200001C01AF2060EE8CFA3F527C200F228C29C
:103F300001F229C202F22AC203F22BC20AF22CC2F7
:103F40000BF22DC20CF22EC20DF223C20EF224C2CD
:103F50000FF225C210F226C211F205EEA4F0EF50C6
:103F6000FE0B0109EF6E0501DF2BB9D044D0EEEC5A
:103F700002F019C202F01AC203F00350015C02E120
:103F80000250005CD8A02DD000D0EEEC02F019C297
:103F9000E8FF005C026E1AC2E8FF0158036E000ED3
:103FA000035C0A0ED8B4025C000ED8B0010E006E9D
:103FB000016A18D0EEEC02F000C002F001C003F07C
:103FC00019C2F6FF1AC2F7FFFF0E006EFF0E016E58
:103FD000F650005EF750015A0250002603500122AD
:103FE00001D0E8D701500010D8B401D001D003D0DF
:103FF000020EE8CFA3F573D0EEEC02F019C202F086
:104000001AC203F00350015C02E10250005CD8A028
:104010002DD000D0EEEC02F019C2E8FF005C026E79
:104020001AC2E8FF0158036E000E035C0A0ED8B4F2
:10403000025C000ED8B0010E006E016A18D0EEECE2
:1040400002F000C002F001C003F019C2F6FF1AC26C
:10405000F7FFFF0E006EFF0E016EF650005EF75088
:10406000015A025000260350012201D0E8D7015026
:104070000010D8B401D001D01AD00201FF0E1B27C6
:10408000FF0E1C23FF0E1D23FF0E1E2302011B51DA
:104090001C111D111E11D8A401D001D002D00501A0
:1040A000A36BEEEC02F000C019F201C01AF217D0B7
:1040B000A3C5E8FF000A01E117D6010A01E14ED6C7
:1040C000030A01E190D6010A01E1A6D6070A01E13F
:1040D000FBD6010A01E10DD7030A8EE000D01200E1
:1040E00002D608D0080EE8CFA3F5E0C5E8FFC1EC82
:1040F00000F01200F7D7C2D10001266B02013C0E7E
:104100001B6F1C6B1D6B1E6B0001280E2D6F000EAC
:104110002E6FBFEC01F000012851020AD8A401D093
:1041200001D081D1276B0F0E275DD8A001D001D01F
:1041300001D00FD00001280E2D6F000E2E6FBFECA6
:1041400001F00001272B0F0E275DD8A001D001D070
:10415000F1D70001270E2D6F020E2E6FBFEC01F07C
:104160000001280E2D6F020E2E6FBFEC01F0000132
:10417000290E2D6F020E2E6FBFEC01F000012A0EEA
:104180002D6F020E2E6FBFEC01F00001276BDC0ECD
:10419000275DD8A001D001D001D00FD00001280E9A
:1041A0002D6F000E2E6FBFEC01F00001272BDC0EEF
:1041B000275DD8A001D001D0F1D70001256B000107
:1041C000280E2D6F000E2E6FBFEC01F012D10001F2
:1041D000280E2D6F000E2E6FBFEC01F00001280598
:1041E000D8A401D001D008D00001260E2D6F000EFA
:1041F0002E6FBFEC01F001D03ED10ED10001280E90
:104200002D6F000E2E6FBFEC01F000012851040A43
:10421000D8A401D001D01DD000012B0E2D6F020EAD
:104220002E6FBFEC01F000012C0E2D6F020E2E6FD1
:10423000BFEC01F000012D0E2D6F020E2E6FBFECB2
:1042400001F000012E0E2D6F020E2E6FBFEC01F05B
:1042500001D011D1E1D00001280E2D6F000E2E6F7C
:10426000BFEC01F0040E0001285DD8A001D001D000
:104270001DD00001230E2D6F020E2E6FBFEC01F03A
:104280000001240E2D6F020E2E6FBFEC01F0000115
:10429000250E2D6F020E2E6FBFEC01F00001260ED1
:1042A0002D6F020E2E6FBFEC01F001D0E4D0FC0E9A
:1042B0000001282707D00001270E2D6F000E2E6F5A
:1042C000BFEC01F0000128072829D8A401D001D0B3
:1042D000F2D7A2D00001280E2D6F000E2E6FBFEC7A
:1042E00001F000012851040AD8A401D001D01DD04A
:1042F00000012C0E2D6F000E2E6FBFEC01F000019F
:104300002B0E2D6F000E2E6FBFEC01F000012A0E58
:104310002D6F000E2E6FBFEC01F00001290E2D6FE6
:10432000000E2E6FBFEC01F001D0A5D075D00001BA
:10433000256B252B71D00001280E2D6F000E2E6FDE
:10434000BFEC01F000012851040AD8A401D001D02B
:1043500037D000011E0E2D6F020E2E6FBFEC01F044
:1043600000011D0E2D6F020E2E6FBFEC01F000013B
:104370001C0E2D6F020E2E6FBFEC01F000011B0E04
:104380002D6F020E2E6FBFEC01F002EE1EF0000E3C
:10439000ED5C08E1000EED5C05E1070EED5C02E16D
:1043A000090EEF5CD8A001D001D009D00201F80EAF
:1043B0001B27F80E1C23FF0E1D23FF0E1E2301D00A
:1043C0005AD02AD00001280E2D6F000E2E6FBFECA0
:1043D00001F007D00001270E2D6F000E2E6FBFECED
:1043E00001F0000128072829D8A401D001D0F2D774
:1043F00013D000012851010A01E100D7020A01E1AE
:104400002AD7300A98E0060A01E1E1D6030A01E161
:1044100061D7C90A8CE0D6D7000125510009D8B46C
:1044200001D001D0CCD600012651020AD8A401D077
:1044300001D009D029C01FF22AC020F22BC021F2DE
:104440002CC022F213D002EE1FF00001EE50291909
:1044500008E1EE502A1905E1EE502B1902E1EE5069
:104460002C19D8B401D001D001D0266BE2EC01F0B8
:104470000001265102D0000E00D012003DD6D8D047
:104480000001256F010ECEEC00F0010ECEEC00F025
:10449000060ECEEC00F0000ECEEC00F0120ECEECCC
:1044A00000F0230ECEEC00F0340ECEEC00F0560EF1
:1044B000CEEC00F0000ECEEC00F0000ECEEC00F0E2
:1044C000800ECEEC00F0000ECEEC00F00001255185
:1044D000030AD8A401D001D014D027C2E8FFCEEC43
:1044E00000F002EE28F0EF50CEEC00F002EE29F0E2
:1044F000EF50CEEC00F002EE2AF0EF50CEEC00F0E0
:104500000CD0000ECEEC00F0000ECEEC00F0000E51
:10451000CEEC00F0000ECEEC00F00001266B00D0D7
:10452000000ECEEC00F00001262B0C0E265DD8A06C
:1045300001D001D0F5D702EE04F0EF50CEEC00F040
:1045400002EE05F0EF50CEEC00F002EE06F0EF5078
:10455000CEEC00F002EE07F0EF50CEEC00F002EEF1
:1045600008F0EF50CEEC00F002EE09F0EF50CEEC88
:1045700000F00001266B00D0000ECEEC00F0000130
:10458000262BCA0E265DD8A001D001D0F5D7630E28
:10459000CEEC00F0820ECEEC00F0530ECEEC00F02C
:1045A000630ECEEC00F0350ECEEC00F0010ECEEC3A
:1045B00000F000012551CEEC00F000012505D8B433
:1045C0000AD000D002012751281129112A11D8B48C
:1045D00002D000D002D000D019D0360ECEEC00F0C0
:1045E000040ECEEC00F002EE22F0EF50CEEC00F024
:1045F00002EE21F0EF50CEEC00F002EE20F0EF5092
:10460000CEEC00F01FC2E8FFCEEC00F0370ECEEC8F
:1046100000F0020ECEEC00F0010ECEEC00F0030E26
:10462000CEEC00F0FF0ECEEC00F020EC01F012001A
:1046300027D7D96AD950006E016AD8900034026E2B
:104640000134036EFA0E0224E96E010E0320EA6EB5
:10465000D9CF00F0D8900036D8900034400FEF6EDC
:10466000D950006E016AD8900034026E0134036E96
:10467000FB0E0224E96E010E0320EA6E010EEF6EBE
:10468000D92AD95CD8A0D6D70501A76BD3DA020EF8
:10469000FBEC34F01F0EEADAE8CFE6F01F0EDADAB0
:1046A000020EFBEC34F0070EE1DA006E00AE1200F1
:1046B000210EE8CFE6F0000ECDDA020EFBEC34F06E
:1046C000480EE8CFE6F00E0EC5DA0001E66B0A0EE2
:1046D000C1DA0001E66B0B0EBDDA040EE8CFE6F09E
:1046E0000C0EB8DA020EE8CFE6F00D0EB3DAA7C56D
:1046F00000F0016AD8900034026E0134036EFA0EA5
:104700000224E96E010E0320EA6EEF50E8CFE6F0D6
:10471000040EA0DA440EE8CFE6F0010E9BDA5F0E3D
:10472000E8CFE6F0020E96DA5E0EE8CFE6F0030E72
:1047300091DAFF0EE8CFE6F0070E8CDA0001E66BA7
:104740000F0E88DA610EE8CFE6F0000E83DA04C2BD
:10475000E6F0010E7FDA05C2E6F0020E7BDA06C251
:10476000E6F0030E77DA07C2E6F0040E73DA08C249
:10477000E6F0050E6FDA09C2E6F0060E6BDA00010C
:10478000156BFF0EE8CFE6F000011551080F62DA55
:104790000001152B080E155DD8A0F3D7440EE8CF05
:1047A000E6F0070E57DA440EE8CFA8F5220EE8CF60
:1047B000E6F0000E4FDA0001E66B0D0E4BD2040E50
:1047C00055DA006E010E016E001412000001E06F58
:1047D000010EE8CFE6F00A0E3DDA0001E66B0B0EA3
:1047E00039DA120EE8CFE6F0000E34DAE0C0E6F077
:1047F000100E30D20001010EE215006E000EE3151E
:10480000016EE2510024E46FE3510120E56F400E98
:10481000E8CFE6F0070E1EDAE4C0E6F00A0E1ADA78
:10482000E5C0E6F00B0E16DA120EE8CFE6F0000E49
:1048300011DA0001E351016EE251006EE207D8A0E7
:10484000E3070110D8B40CD0E0C0E9FFE1C0EAFFF3
:10485000EF50E8CFE6F0E04BE12B100EFBD9E9D7A3
:10486000FF0E0001E26FE36B0001E351E211D8B4E7
:104870001200070EFBD9006E00BC12000001E20717
:10488000D8A0E307F1D7010EE8CFE6F00A0EE2D98F
:104890000001E66B0B0EDED90A0EE8CFE6F0000E43
:1048A000D9D9100EE3D157C059F058C05AF0400E74
:1048B000E8CFE6F0070ECED959C0E6F00A0ECAD905
:1048C0005AC0E6F00B0EC6D90A0EE8CFE6F0000E8D
:1048D000C1D900015851016E5751006E5707D8A039
:1048E00058070110D8B40BD0100EC0D955C0E9FF3D
:1048F00056C0EAFFEF6E0001554B562BEAD759C060
:1049000000F05AC001F01200D96E006E016AD89012
:104910000034026E0134036EFB0E0224E96E010EB8
:104920000320EA6E000EEF6A1200D96E006E016A73
:10493000D8900034026E0134036EFB0E0224E96E3F
:10494000010E0320EA6E010EEF6ED9CFA7F512001B
:10495000A8C500F000040001806F440E805DD8B04F
:1049600002D05E0E806F200EE8CFE6F0000E72D906
:1049700080C0E6F0030E6ED1600EE8CFE6F0000EC8
:1049800069D9070E73D90001BF6F200EE8CFE6F09A
:10499000000E60D90001A6C5E8FFBF5DA6C5E8FF0F
:1049A000D8B005D05F08006EBF51002402D00001CE
:1049B000BF5DD96E1B08D96ED9CFC1F00001C06BA5
:1049C000C0C000F0C1C001F012001B001DC0E9FF13
:1049D0001EC0EAFFFF0EEF6E070E48D9006E00A85A
:1049E00024D0210EE8CFE6F0000E34D9FF0E5BD9BB
:1049F0000001E66B0A0E2ED90001E66B0B0E2AD9D8
:104A0000020EE8CFE6F00D0E25D9200EE8CFE6F035
:104A1000000E20D99DDFFF0EE8CFE6F0070E1AD971
:104A20000001E66B0D0E16D9000C600EE8CFE6F023
:104A3000000E10D9070E1AD900011F6F200EE8CF03
:104A4000E6F0000E07D9A8C500F000011F510018BC
:104A5000D8B4000CA8C521F0206B20C0E0F021C024
:104A6000E1F010D90001220E556F000E566F0001C3
:104A7000120E576F586B17DF22A13DD00001000EB8
:104A8000255D400ED8B4245DD8A035D0050E255D37
:104A9000EF0ED8B4245DD8B02ED032C0DAF033C0D7
:104AA000DBF0DFEC2CF000C032F001C033F01BC0B3
:104AB0005BF01CC05CF000012C0E5D6F000E5E6FA1
:104AC0000001060E5F6F606B68EC34F033C0E8FFE6
:104AD000080AD8A410D000EE32F0EF50D8B405D0B8
:104AE00032C0E8FF060AD8A406D01DC0E9FF1EC0E8
:104AF000EAFF32C0EFFFA8C5A6F523C0A8F5010C58
:104B0000D8000A0EE8CFE6F0070EA4D8A7C500F03B
:104B1000016AD8900034026E0134036EFA0E02244A
:104B2000E96E010E0320EA6EEF50E8CFDFF00001DE
:104B3000DE6BDEC0E0F0DFC0E1F0A4D8D8C0E0F06A
:104B4000D9C0E1F00001060EE26FE36B53DE02EE26
:104B500004F0EF503BDE02EE05F0EF5037DE02EEE0
:104B600006F0EF5033DE02EE07F0EF502FDE02EEDC
:104B700008F0EF502BDE02EE09F0EF5027DE0001C7
:104B8000DA51D8A402D0DD6B03D00001060EDD6F30
:104B9000080E1CDE0001DD5119DE0E0E0001DB27C0
:104BA000000EDC23DC5D3C0ED8B4DB5DD8B003D056
:104BB000400EDB6FDC6BDBC0DEF0DCC0DFF0DEC0A4
:104BC000E6F0050E47D8DFC0E6F0060E43D0A7C5D5
:104BD00000F0016AD8900034026E0134036EFA0EC0
:104BE0000224E96E010E0320EA6EEF50E8CFE6F0F2
:104BF000040E30D8240EE8CFE6F0000E2BD8D96A88
:104C0000D950006E016AD8900034026E0134036EF0
:104C1000FB0E0224E96E010E0320EA6EEF50D8B4B9
:104C200003D0D9CFA7F51200D92A010ED95CD8B08C
:104C30001200E6D79568816AE00E936EF19E848239
:104C400084808484966AD96AD92AD92EFED784941E
:104C50001200E600D96E816EE00E936E0001E651FF
:104C6000836E956A8492848295681200E16E9568DD
:104C7000E150816EE00E936E84908350D96E8480F3
:104C80001200E000E0C0E2F0E1C0E3F0400EE8CF47
:104C9000E6F0070EDFDFE2C0E6F0080EDBDFE3C080
:104CA000E6F0090ED7D70001356F346B000135519E
:104CB000016E3451006E3407D8A035070110D8B406
:104CC0001200F4D7A6C582F0120EE8CF81F00001E1
:104CD0007F5181278051822381C0E0F082C0E1F0C2
:104CE000D1D7E16EE1CFA7F5A7C500F0016AD89052
:104CF0000034026E0134036EFA0E0224E96E010ED6
:104D00000320EA6EEF50E8CFC2F00E0EE8CFC1F0FC
:104D10000001BF51C127C051C223C1C0E0F0C2C0D1
:104D2000E1F042EF26F03F0000014D6B4E6B3FC0BB
:104D30004BF040C04CF0000143C0F6FF44C0F7FF09
:104D4000010E4327000E4423050EF76403D008002C
:104D5000F55005D0F6CFE9FFF7CFEAFFEF50486FE7
:104D600000090001D8B4D1D2250AD8B40AD04D4BDD
:104D70004E2B42514111D8A484D1485103EC00F08C
:104D8000DAD700014669476B456B6CD2000142518E
:104D90004111D8B406D041C0E9FF42C0EAFF000E7D
:104DA000EF6A4DC000F04EC001F0120000014C51FE
:104DB000016E4B51006E020E4B27D8B04C2B00C039
:104DC000E9FF01C0EAFFEFCF47F04CD20001458D6B
:104DD00049D20001452B06D0080E00014627FE0EE1
:104DE0000001462700014C51016E4B51006E020E2E
:104DF0004B27D8B04C2B00C0E9FF01C0EAFFEECF33
:104E000049F0EDCF4AF045A10ED04AAF07D0491F77
:104E10004A1F492BD8B44A2B470707D000014591B8
:104E200045AD03D0F9D7000145910B0E000146278F
:104E30004651026E036A49C000F04AC001F09FEC7F
:104E400034F00050486F4651026E036A49C000F0CA
:104E50004AC001F09FEC34F004C049F005C04AF0AC
:104E6000010E4F6F506B000150514A5D02E14F51EE
:104E7000495DD8A010D000014651026E036A4FC0B0
:104E800000F050C001F016EC35F004C04FF005C042
:104E900050F04707E8D745A914D01AD000014D4B70
:104EA0004E2B42514111D8B409D041C0E9FF42C054
:104EB000EAFF200EEF6E414B422B03D0200E03EC95
:104EC00000F0000147074751800A7F0FD8B0E6D7AE
:104ED00045A114D000014D4B4E2B42514111D8B485
:104EE00009D041C0E9FF42C0EAFF2D0EEF6E414BF1
:104EF000422B16D02D0E03EC00F012D045AD10D091
:104F000000014D4B4E2B42514111D8B406D041C047
:104F1000E9FF42C0EAFF2B0EE9D72B0E03EC00F0AD
:104F200045B914D04DD000014D4B4E2B425141118B
:104F3000D8B409D041C0E9FF42C0EAFF300EEF6E9D
:104F4000414B422B03D0300E03EC00F00001470729
:104F50004751800A7F0FD8A033D0E5D74FC002F069
:104F600050C003F049C000F04AC001F09FEC34F09B
:104F700004C000F005C001F000014651026E036A52
:104F80009FEC34F00050476F800A760FD8A002D013
:104F9000070E472700014D4B4E2B42514111D8B40B
:104FA0000AD04751300F41C0E9FF42C0EAFFEF6E1F
:104FB000414B422B05D000014751300F03EC00F06C
:104FC00000014651026E036A4F0EE96E000EEA6E52
:104FD000EE50006EEF50016E9FEC34F00550ED6E18
:104FE0000450EF6EEE50ED10D8A4B8D70A0E0001B1
:104FF000485DD8A002D0070E482700014D4B4E2B2C
:1050000042514111D8B408D04851300F41C0E9FF96
:1050100042C0EAFFEF6E3BD000014851300F03EC75
:1050200000F089D600014751800A7E0FD8A015D024
:105030004D4B4E2B42514111D8B409D041C0E9FF2C
:1050400042C0EAFF200EEF6E414B422B03D0200EF0
:1050500003EC00F000014707E5D74C51016E4B51BE
:10506000006E020E4B27D8B04C2B00C0E9FF01C0E8
:10507000EAFFEFCF48F04D4B4E2B42514111D8B4CF
:1050800009D041C0E9FF42C0EAFF48C0EFFF414BF1
:10509000422B51D60001485103EC00F04CD60001E0
:1050A0004C51016E4B51006E020E4B27D8B04C2B69
:1050B00000C0E9FF01C0EAFFEECF00F0EDCF01F044
:1050C00000C013F001C014F0D96AD950006E016A13
:1050D00013C0E8FF0024026E14C0E8FF0120036E35
:1050E00002C0F6FF03C0F7FF050EF76403D0080007
:1050F000F55005D0F6CFE9FFF7CFEAFFEF500009F2
:10510000D8B402D0D92AE1D700014651D95CD8B031
:1051100002D0D950466F0001465147BF42D0FF0A26
:105120004725D8A03FD04D4B4E2B42514111D8B40A
:1051300009D041C0E9FF42C0EAFF200EEF6E414BAB
:10514000422B03D0200E03EC00F000014707E3D709
:1051500013C0F6FF14C0F7FF050EF76403D0080074
:10516000F55005D0F6CFE9FFF7CFEAFFEF50000189
:10517000486F0001132B000E142300014D4B4E2BE2
:1051800042514111D8B409D041C0E9FF42C0EAFF01
:1051900048C0EFFF414B422B04D00001485103ECC3
:1051A00000F0000146074629D8B4C5D5D1D743C081
:1051B000F6FF44C0F7FF050EF76403D00800F55072
:1051C00005D0F6CFE9FFF7CFEAFFEF502A0AD8A4BF
:1051D00012D000014C51016E4B51006E020E4B2754
:1051E000D8B04C2B00C0E9FF01C0EAFFEFCF46F07A
:1051F000434B442B37D043C0F6FF44C0F7FF050EA6
:10520000F76403D00800F55005D0F6CFE9FFF7CFDB
:10521000EAFFEF50D00F0001466F434B442B43C0D1
:10522000F6FF44C0F7FF050EF76403D00800F55001
:1052300005D0F6CFE9FFF7CFEAFFEF50D96E300E79
:10524000D95CD8A00FD03A0ED95CD8B00BD046515B
:105250000A0DD950F324D00F466FCAD745B539D0BF
:1052600000014589000143C0F6FF44C0F7FF010E6D
:105270004327000E4423050EF76403D00800F550C1
:1052800005D0F6CFE9FFF7CFEAFFEF50486F000AED
:1052900001E17CD52A0A01E189D5010A01E196D50F
:1052A000050A85E01E0ADAE0680A01E195D53B0AA5
:1052B00001E1B8D6070A01E18CD50B0A01E18FD5CF
:1052C0001C0A01E1ECD6060A01E18CD50D0A01E1C8
:1052D00083D5300E0001485DD8A00CD03A0E485D51
:1052E000D8B008D0458547510A0D4851F324D00F56
:1052F000476FB8D700014D4B4E2B42514111D8A4F6
:10530000C0D6485103EC00F016D542514111D8B433
:1053100006D041C0E9FF42C0EAFF000EEF6A4DC06F
:1053200000F04EC001F01200260090D000012A0EBD
:10533000556F000E566F00011C0E576F586B53ECE3
:1053400024F0A8EC24F000012A0E466F000E476FEF
:105350005CD900012A51010A2B11D8B401D006D022
:105360002EC0E8FF060AD8B402D000D007D000D083
:105370002FC0E8FF040AD8B402D000D002D000D079
:1053800002D0000E62D028C0E1FF29C0E2FF26C093
:10539000D9FF27C0DAFF00013051020A3111D8A429
:1053A00001D001D003D0000EE76E0FD000013051C4
:1053B000010A3111D8A401D001D003D0010EE76E4B
:1053C00004D0020EE76E000E40D000C2E8FF0001DC
:1053D000426308D000D002EE01F0EF50436302D0E8
:1053E00000D001D007D002EE02F0EF50446302D0AB
:1053F00000D001D007D002EE03F0EF50456302D099
:1054000000D002D000D01FD0320E006E000E016E10
:1054100000C0E9FF01C0EAFFD9CFE1FFDACFE2FF28
:10542000060E51EC35F000EE06F0D950E926DA50C0
:10543000EA2238C0EEFF39C0EEFF3AC0EEFF3BC0B3
:10544000EEFF010E02D0000E00D012006FD7260032
:10545000DAD026C0D9FF27C0DAFF0001010E296F7C
:105460002A6B0001000E2B6F080E2C6F060EE8CF82
:105470002DF0040EE8CF2EF000012805D8A401D0AD
:1054800001D017D00001010E2F6F306BFF0EE8CF57
:105490003BF0FF0EE8CF3CF0FF0EE8CF3DF0FF0EF3
:1054A000E8CF3EF0FF0EE8CF3FF0FF0EE8CF40F030
:1054B00013D00001020E2F6F306BD9CF00F0DACF7E
:1054C00001F000C0E9FF01C0EAFF3B0EE16E000EF3
:1054D000E26E060E51EC35F004C231F005C232F036
:1054E00006C233F007C234F008C235F009C236F004
:1054F00000C237F001C238F002C239F003C23AF0FC
:105500000AC200F000EE06F0D950E926DA50EA228D
:10551000EF50016E0001015037190014D8B401D0CA
:1055200010D00BC200F000EE07F0D950E926DA5097
:10553000EA22EF50016E015038190014D8B402D09D
:1055400000D011D000D00CC200F000EE08F0D9500D
:10555000E926DA50EA22EF50016E015039190014A1
:10556000D8B402D000D011D000D00DC200F000EEAF
:1055700009F0D950E926DA50EA22EF50016E0150C5
:105580003A190014D8B402D000D002D000D009D00B
:105590000EC241F00FC242F010C243F011C244F0FB
:1055A00010D000EE06F0D950E926DA50EA22EECF0C
:1055B00041F0EECF42F0EECF43F0EDCF44F0ED52AC
:1055C000ED520001290E466F000E476F1ED80001F4
:1055D0003B0ED86F000ED96F060EE8CFDAF000014F
:1055E0001C0EDB6FDC6B81EC25F00001290EE06FF7
:1055F000000EE16F00011C0EE26FE36BFAEC23F08A
:10560000E7EC25F0120025D746004ED046C0E9FF52
:1056100047C0EAFFEECF00F0EDCF01F000C0DAF0B6
:1056200001C0DBF0DFEC2CF046C0E9FF47C0EAFF29
:1056300000C0EEFF01C0EDFF000100EE02F0465198
:10564000E9264751EA22EECF00F0EDCF01F000C08D
:10565000DAF001C0DBF0DFEC2CF0000100EE02F02C
:105660004651E9264751EA2200C0EEFF01C0EDFF96
:1056700000EE06F04651E9264751EA22EECF00F04F
:10568000EDCF01F000C0DAF001C0DBF0DFEC2CF070
:10569000000100EE06F04651E9264751EA2200C01B
:1056A000EEFF01C0EDFF1200B1D71B000001400E5C
:1056B000556F000E566F0001140E576F586B53EC68
:1056C00024F0F00E006E00014015400AD8A4B3D0BB
:1056D00040C000F00F0E0016D8900036D89000346D
:1056E000EC0F236F150E235DD8B0A5D02351D8B48D
:1056F0000CD000012C0E556F000E566F0001235187
:105700000001576F586B53EC24F000EE4AF0EECFD7
:1057100026F0EDCF27F000014A6B4B6B0001400EE5
:10572000D86F000ED96F0001140EDA6FDB6B46ECF8
:105730002DF0001C026E011C036E02C028F003C095
:1057400029F000012351D8B415D000012C0ED86FD8
:10575000000ED96F000123510001DA6FDB6B46ECBC
:105760002DF0001C026E011C036E02C02AF003C063
:105770002BF003D000012A6B2B6B0001280ED86F91
:10578000000ED96F0001040EDA6FDB6B46EC2DF0D2
:1057900000C024F001C025F00001400ED86F000EBB
:1057A000D96FB9D800012551271902E124512619D2
:1057B000D8A441D0F00E006E4015400AD8A43BD0CA
:1057C0001BC0E1FF1CC0E2FFE250E110D8B40CD0D6
:1057D000E1CFE9FFE2CFEAFF50C0EEFF51C0EEFF9C
:1057E00052C0EEFF53C0EEFF000100EE06F01D5167
:1057F000E9261E51EA224CC0EEFF4DC0EEFF4EC01E
:10580000EEFF4FC0EEFF1FC0E9FF20C0EAFF49C016
:10581000EFFF2351425D006E4351D8A04305016E56
:10582000EC0E002421C0E9FF22C0EAFFEE6EFF0E5D
:105830000120ED6E010CA8EC24F0000CBF00450E19
:10584000E8CFC4F00001C56B140EC225E8CFC6F046
:10585000000EC321E8CFC7F00001112B000E122368
:1058600011C0C8F012C0C9F00001CA6BCB6B640E46
:10587000E8CFCCF0C1C0CDF0CE6BCF6B00C2D0F082
:1058800001C2D1F002C2D2F003C2D3F000EE06F0A2
:10589000BF51E926C051EA22EECFD4F0EECFD5F0C9
:1058A000EECFD6F0EDCFD7F0ED52ED520001C40EA1
:1058B000D86F000ED96F2FD80001C40ED86F000E1C
:1058C000D96F0001140EDA6FDB6B46EC2DF000C0CF
:1058D000CEF001C0CFF0BFC0D8F0C0C0D9F00001F9
:1058E000DA6B0001140EC225E8CFDBF0000EC321F5
:1058F000E8CFDCF081EC25F00001C40EE06F000E73
:10590000E16F0001140EE26FE36BFAEC23F0006A22
:10591000016A1200D800000100EE02F0D851E92619
:10592000D951EA22EECF00F0EDCF01F000C0DAF05D
:1059300001C0DBF0DFEC2CF0000100EE02F0D851EA
:10594000E926D951EA2200C0EEFF01C0EDFF00EECA
:1059500004F0D851E926D951EA22EECF00F0EDCF7C
:1059600001F000C0DAF001C0DBF0DFEC2CF0000148
:1059700000EE04F0D851E926D951EA2200C0EEFF2A
:1059800001C0EDFF00EE0AF0D851E926D951EA2214
:10599000EECF00F0EDCF01F000C0DAF001C0DBF097
:1059A000DFEC2CF0000100EE0AF0D851E926D951C5
:1059B000EA2200C0EEFF01C0EDFF1200DA0012D0B3
:1059C000DAC0DCF0DBC0DDF000EEDDF0EFCFDEF0C2
:1059D000DCC0DDF0DEC0DCF0DCC000F0DDC001F0DA
:1059E00000D01200EDD7C1004FD0C1C0C6F0C2C078
:1059F000C7F0C3C0C8F0C4C0C9F00001C60ECA6F6A
:105A0000000ECB6F00EE03F0CA51E926CB51EA221B
:105A1000EFCFC5F0CAC0E9FFCBC0EAFF10EE03F03C
:105A2000CA51E126CB51E222EFCFE7FFCAC0E9FF1E
:105A3000CBC0EAFFC5C0EFFF00EE02F0CA51E92675
:105A4000CB51EA22EFCFC5F010EE01F0CA51E126AA
:105A5000CB51E22200EE02F0CA51E926CB51EA22F4
:105A6000E7CFEFFF00EE01F0CA51E926CB51EA2261
:105A7000C5C0EFFFC6C000F0C7C001F0C8C002F04B
:105A8000C9C003F000D01200B0D7D80084D0000104
:105A9000E46BE56BE66BE76BD890DB31DD6FDA31F9
:105AA000DC6FD8C0DEF0D9C0DFF01BD00001DF51C1
:105AB000016EDE51006E020EDE27D8B0DF2B00C073
:105AC000E9FF01C0EAFFEECF00F0EDCF01F0026A7E
:105AD000036A0050E4270150E5230250E6230350F7
:105AE000E7230001DD51016EDC51006EDC07D8A018
:105AF000DD0701500010D8A401D001D0D7D7DAA11A
:105B000001D001D00ED0DEC0E9FFDFC0EAFFEF50C8
:105B10000001E427010ED8B0E527D8B0E627D8B0B9
:105B2000E727E4C0E0F0E5C0E1F0E6C0E2F0E7C05E
:105B3000E3F01DD00001E66BE76BE451DC25006E5D
:105B4000E551DD21016E026AD8B0022A036A00C065
:105B5000E4F001C0E5F002C0E6F003C0E7F0E4C005
:105B6000E0F0E5C0E1F0E6C0E2F0E7C0E3F000EE0F
:105B7000E2F0EECFDCF0EDCFDDF00001DD51DC1125
:105B8000D8A401D001D0D6D70001E41D006EE51DD8
:105B9000016E00D012007BD78F002ED08FC092F004
:105BA00090C093F017D0610E0001915DD8A007D08E
:105BB00000D07B0E915DD8B002D000D002D000D0D2
:105BC00006D092C0E9FF93C0EAFFE00EEF26000185
:105BD000924B932B92C0E9FF93C0EAFFEF50000174
:105BE000916F0009D8A401D001D0DDD78FC000F09B
:105BF00090C001F000D01200D1D78F002FD091C0FB
:105C000096F092C097F08FC094F090C095F019D0A4
:105C100096C0F6FF97C0F7FF94C0E9FF95C0EAFF72
:105C2000050EF76403D00800F55005D0F6CFE1FF6C
:105C3000F7CFE2FFE750EF6E0001944B952B964BA8
:105C4000972B000193079329D8A401D001D0E0D766
:105C50008FC000F090C001F000D01200D0D7050135
:105C6000AC6B05EEADF0EF50FE0B0109EF6E19ECD9
:105C700023F021EC34F04EEC00F0F4EF08F00001DA
:105C8000156B152B00011551D8B423D1156B09D113
:105C90000001350E1B6F020E1C6F0001160E1D6FEA
:105CA000000E1E6FE6EC24F0006E016A0150001039
:105CB0000001D8B4E8D7156B152B1651D8A402D023
:105CC000020E61D000011651060AD8A402D0050EBA
:105CD0005AD0A8EC24F0D6D70001156B26EC34F08E
:105CE0000009D8B4CFD756D00001170E1B6F000E95
:105CF0001C6F0001350E1D6F020E1E6F0001160E87
:105D00001F6F000E206F00012F0E216F020E226FF9
:105D100056EC2BF0006E016A01500010D8B43DD053
:105D20000001156B152B1605D8A420D0030EE8CF63
:105D3000ACF5ADC500F000A0A5D71729D8B4182937
:105D4000D8B41929D8B41A29D8B49CD705EEADF027
:105D5000EF50FE0BEF6E17C000F218C001F219C031
:105D600002F21AC003F271EC20F08CD70001165138
:105D7000060AD8A402D0060E06D000011651110A58
:105D8000D8A404D0070EE8CFACF57CD70001156B82
:105D9000A8EC24F00501AC6B75D7A8EC24F0FAD779
:105DA0000001350E1B6F020E1C6F2FC21DF030C29A
:105DB0001EF0FEEC01F0006E016A01500010D8B434
:105DC00002D00501AC6B0001156B5CD70001350EEC
:105DD0001B6F020E1C6F2FC21DF030C21EF09BEC19
:105DE0000CF0006E016A01500010D8A4EAD7EBD77E
:105DF0000501AC6B0201000E305D2A0ED8B42F5D98
:105E0000D8B02ED00001160E1B6F000E1C6F0001C3
:105E1000AE0E1D6F050E1E6F00012F0E1F6F020EBE
:105E2000206F0001310E216F020E226F0001330E30
:105E3000236F020E246F78EC2FF0006E016A015080
:105E40000010D8B40BD000011651080AD8A406D00F
:105E5000156B152B040EE8CFACF502D00501AC6B29
:105E6000A8EC24F00FD7DFEC23F00009D8B40AD750
:105E70000001350E1B6F020E1C6F00011D6B00012F
:105E8000AE0E1E6F050E1F6F2FC220F031C221F023
:105E900032C222F033C223F034C224F0FBEC2FF0E4
:105EA00079D7ACC5E8FF000A01E1F2D6010A01E1A9
:105EB000EFD6030A01E118D7010A9AE0070AD3E0F6
:105EC000010A01E109D7030A81E0010A01E168D76B
:105ED000D9D699EC0CF072EC1EF0A4C500F000A02D
:105EE000120005EEADF0EF50FE0BEF6E12001B003E
:105EF00000012D0E556F000E566F0001080E576FF2
:105F0000586B53EC24F000EE2FF0EECF27F0EDCFDE
:105F100028F000012F6B306B00012D0ED86F000EA2
:105F2000D96F0001080EDA6FDB6B46EC2DF0001C18
:105F3000026E011C036E02C029F003C02AF01FC0CC
:105F4000E1FF20C0E2FFF80EE7261DC055F01EC09D
:105F500056F0E7500001576F586B53EC24F01DC00A
:105F6000D8F01EC0D9F01FC0E9FF20C0EAFFEF50F3
:105F70000001DA6FDB6B46EC2DF0001C026E011C99
:105F8000036E02C02BF003C02CF00001290ED86F65
:105F9000000ED96F0001040EDA6FDB6B46EC2DF0BA
:105FA00000C025F001C026F000012D0E556F000E37
:105FB000566F86D81BC0E9FF1CC0EAFF2DC0EFFF5B
:105FC00021C0E9FF22C0EAFF31C0EEFF32C0EDFF81
:105FD00023C0E9FF24C0EAFF33C0EEFF34C0EDFF69
:105FE00000012851261902E127512519000ED8B4C5
:105FF000010E12001B000001266B1DC025F0276B4F
:10600000286B21C029F022C02AF023C02BF024C025
:106010002CF000012D0E5B6F000E5C6F1EC05DF05A
:106020001FC05EF00001205100015F6F606B68ECE3
:1060300034F00001250E556F000E566F41D8000157
:10604000250ED86F000ED96F00012051006E016A35
:10605000080E0024E8CFDAF0000E0120E8CFDBF0D4
:1060600046EC2DF000C027F001C028F01BC0BFF0A7
:106070001CC0C0F0010EE8CFC1F000012051006E3D
:10608000016A080E0024E8CFC2F0000E0120E8CF1C
:10609000C3F01FEC2CF00001250EE06F000EE16F45
:1060A00000012051006E016A080E0024E8CFE2F0E2
:1060B000000E0120E8CFE3F0FAEC23F0E7EF25F043
:1060C000000100EE04F05551E9265651EA22EECFC8
:1060D00000F0EDCF01F000C0DAF001C0DBF0DFEC42
:1060E0002CF0000100EE04F05551E9265651EA2249
:1060F00000C0EEFF01C0EDFF00EE06F05551E926AD
:106100005651EA22EECF00F0EDCF01F000C0DAF0F8
:1061100001C0DBF0DFEC2CF0000100EE06F0555181
:10612000E9265651EA2200C0EEFF01C0EDFF00EE65
:1061300002F05551E9265651EA22EECF00F0EDCF9C
:1061400001F000C0DAF001C0DBF0DFEC2CF0000160
:1061500000EE02F05551E9265651EA2200C0EEFF4A
:1061600001C0EDFF120007D00501AB6B0501AA6B62
:10617000010E00D01200F8D77B0098D0AAC500F01D
:1061800000A001D001D003D0006A016A8ED00001C6
:10619000AE0E8C6F0E0E8D6F7BC0E9FF7CC0EAFFE8
:1061A000EF50D8A401D001D005D0FF0E006EFF0E35
:1061B000016E7BD07BC08FF07CC090F0CDEC2DF0D9
:1061C00000C07BF001C07CF06AD000017D0E8F6FB3
:1061D000000E906F8CC091F08DC092F00F0EE8CF42
:1061E00093F0FEEC2DF000EE7DF0EF50D8A401D03E
:1061F00001D036D07BC08FF07CC090F0D3EC34F06F
:10620000005000018E6F0D0E8E5DD8A001D001D020
:1062100002D00C0E8E6F7BC08FF07CC090F000011E
:10622000800E916F000E926F00018E510001936FEE
:10623000946B62EC33F001500010D8A401D001D06F
:1062400009D00501AB2B00EE7EF0EECF00F0EDCFD4
:1062500001F02BD00F0E00018C27000E8D231FD0D4
:106260007DC0E8FF040AD8A401D001D013D00001FA
:106270007F51FF0AFF0ED8B47E19D8B401D001D0E7
:1062800007D000EE7EF0EECF8CF0EDCF8DF001D098
:1062900007D005D0FF0E006EFF0E016E06D095D719
:1062A000FF0E006EFF0E016E00D0120067D711D0F6
:1062B0000501A96B05EEAAF0EF50FE0BEF6EABC522
:1062C000E8FF0009D8B401D001D002D00501AB0726
:1062D0001200EED741D0FCC1F6FFFDC1F7FF050E5D
:1062E000F76403D00800F55005D0F6CFE9FFF7CFEB
:1062F000EAFFEF5000017F6F0101FC2B000EFD2330
:1063000000017F51030AD8A401D001D015D0FCC1EF
:10631000F6FFFDC1F7FF050EF76403D00800F55046
:1063200005D0F6CFE9FFF7CFEAFFEF507F6F01010D
:10633000FC2B000EFD230CD000017F51040AD8A4D1
:1063400001D001D005D0FF0EE8CFFCF1E8CFFDF180
:1063500000017F5100D01200BED70BD005EEAAF08D
:10636000EF50FE0B0109EF6E200E006E016A00D0A7
:106370001200F4D705D00001156F010E00D01200F5
:10638000FAD706D0FCC100F0FDC101F000D0120028
:10639000F9D739D0F00E83160F0E9512959A95986D
:1063A000929A839A8398809A65EC1EF0F00E951667
:1063B000F00E83168382808A6BEC1EF0809A68EC64
:1063C0001EF0F00E83168382808A6BEC1EF0809A9A
:1063D0006BEC1EF0F00E83168382808A6BEC1EF04D
:1063E000809A0F0E9512280E0FD8280E0DD8080E81
:1063F0000BD80C0E09D8010E07D8130E05D8800E45
:1064000003D800D01200C6D72DD000013F6F00D0B6
:106410002AD80009D8A401D001D0FAD7959A959826
:10642000F00E9516F00E831600013F390F0B831204
:10643000839A83986BEC1EF0808A6BEC1EF0809A36
:10644000F00E83160F0E006E000100503F158312F0
:106450006BEC1EF0808A6BEC1EF0809A0F0E95128A
:1064600000D01200D2D723D0838A8398959A95982A
:106470006BEC1EF0808A6BEC1EF083A601D001D07D
:106480000BD0809A6BEC1EF0808A6BEC1EF0809A29
:10649000839A010E0BD00AD0809A6BEC1EF0808A92
:1064A0006BEC1EF0809A839A000E00D01200DCD7AD
:1064B0003F0014D006D00001415132D800013F4BBB
:1064C000402B3FC0E9FF40C0EAFFEF500001416FA1
:1064D0000009D8A401D001D0EED71200EBD73F00BD
:1064E0001ED006D0000141511BD800013F4B402B6C
:1064F0003FC0F6FF40C0F7FF050EF76403D0080069
:10650000F55005D0F6CFE9FFF7CFEAFFEF500001D5
:10651000416F0009D8A401D001D0E4D71200E1D71F
:1065200033D00001426F00D09EDF0009D8A401D013
:1065300001D0FAD7959A9598F00E9516F00E83161D
:106540000F0E006E42C001F0013A0F0E011600500E
:10655000011483128388839A6BEC1EF0808A6BECA3
:106560001EF0809AF00E83160F0E006E0001005090
:10657000421583126BEC1EF0808A6BEC1EF0809A41
:106580000F0E951200D01200CCD7390003D00001B5
:10659000394B3A2B39C0F6FF3AC0F7FF050EF764C6
:1065A00003D00800F55005D0F6CFE9FFF7CFEAFF9A
:1065B000EF50200AD8B4EBD739C0F6FF3AC0F7FF46
:1065C000050EF76403D00800F55005D0F6CFE9FFBB
:1065D000F7CFEAFFEF50090A0001D8B4D9D73C6BD6
:1065E0003D6B3B6B39C0F6FF3AC0F7FF050EF76411
:1065F00003D00800F55005D0F6CFE9FFF7CFEAFF4A
:10660000EF502D0AD8A402D03B2B13D039C0F6FF8F
:106610003AC0F7FF050EF76403D00800F55005D027
:10662000F6CFE9FFF7CFEAFFEF502B0AD8A403D04B
:106630000001394B3A2B39C0F6FF3AC0F7FF050E7F
:10664000F76403D00800F55005D0F6CFE9FFF7CF87
:10665000EAFFEF5032EC35F0D8A025D00A0E026EDA
:10666000036A3CC000F03DC001F016EC35F039C0C3
:10667000F6FF3AC0F7FF050EF76403D00800F550A7
:1066800005D0F6CFE9FFF7CFEAFFEF500424006E04
:10669000000E0520016ED00E002400013C6FFF0E9D
:1066A00001203D6FC6D700013B513CC000F03DC00A
:1066B00001F0D8B41200001E011E002AD8B4012A2D
:1066C00012008F0000019451016E9351006E9307E8
:1066D000D8A094070110D8B45ED08FC0F6FF90C048
:1066E000F7FF050EF76403D00800F55005D0F6CF8C
:1066F000E9FFF7CFEAFFEF500009D8B422D091C0EC
:10670000F6FF92C0F7FF050EF76403D00800F550BE
:1067100005D0F6CFE9FFF7CFEAFFEF50006E8FC04C
:10672000F6FF90C0F7FF050EF76403D00800F550A0
:1067300005D0F6CFE9FFF7CFEAFFEF500018D8B445
:1067400024D08FC0F6FF90C0F7FF050EF76403D08A
:106750000800F55005D0F6CFE9FFF7CFEAFFEF507C
:10676000006E016A91C0F6FF92C0F7FF050EF76454
:1067700003D00800F55005D0F6CFE9FFF7CFEAFFC8
:10678000EF50005E000E015A120000018F4B902B5B
:10679000914B922B97D7006A016A12008B008BC035
:1067A00002F08CC003F08DC0F3FF8EC0F4FF000137
:1067B0009051016E8F51006E8F07D8A09007011085
:1067C000D8B43CD0F3CFF6FFF4CFF7FF010EF32699
:1067D000000EF422050EF76403D00800F55005D032
:1067E000F6CFE9FFF7CFEAFFEF50016E02C0F6FFE8
:1067F00003C0F7FF010E0226000E0322050EF76408
:1068000003D00800F55005D0F6CFE9FFF7CFEAFF37
:10681000EF50006E0150005C0001916F926BD8A0A8
:10682000920700BE920701BE922B92519111D8B4EB
:10683000BED791C000F092C001F01200006A016A58
:10684000120003D00501A56B1200FCD73FD036D053
:1068500000011C0E266F000E276F00011B0E286F13
:10686000000E296F95EC29F0006E016A01500010AE
:10687000D8A401D001D001D026D000011B510009BD
:10688000D8A401D001D001D01ED0010EE8CFA5F5CB
:10689000DFEC23F00009D8B401D001D00CD0000106
:1068A0001C0E266F000E276F0001286B28EC2AF0C3
:1068B0000501A56B02D0000E08D005D0A5C5E8FFE4
:1068C000000AC6E0E5D7010E00D01200C0D75B0079
:1068D0005DC0F3FF5EC0F4FF5BC0D9FF5CC0DAFFB0
:1068E00000016051016E5F51006E5F07D8A0600724
:1068F0000110D8B41FD0F3CFF6FFF4CFF7FF010E8D
:10690000F326000EF422DA50016ED950006ED94AF7
:10691000DA2A00C0E9FF01C0EAFF050EF76403D0E0
:106920000800F55005D0F6CFE1FFF7CFE2FFE750C2
:10693000EF6ED6D75BC000F05CC001F01200066AB3
:10694000046A056A0250031003E1006A016A000C40
:106950001F0E0612D890062A02360336FCE30332D5
:1069600002320250005C0350015804E3016E0250F1
:10697000005ED88004360536062E06BAF0D706AE7D
:1069800005D0041E042AD8B40506051E0450026E64
:106990000550036E06AC000C001E002AD8B4010698
:1069A000011E000C8F008FC0F3FF90C0F4FFF3CFE7
:1069B000F6FFF4CFF7FF010EF326000EF422050ECA
:1069C000F76403D00800F55005D0F6CFE9FFF7CF04
:1069D000EAFFEF500009D8A4EAD700018F51F35C19
:1069E000006E9051F458016EFF0E0024006EFF0EF1
:1069F0000120016E120019D0E96E10D0040EE16E74
:106A000007D0500ED96E00D001D000D0D92EFDD7BE
:106A1000E106E128D8A401D001D0F3D7E906E9289E
:106A2000D8A401D001D0EAD71200E6D70250000264
:106A3000F3CF04F0F4CF05F00102F3500526035024
:106A40000002F35005261200EFCF00F0EE2AEFCF40
:106A500001F0000EEE22EFCF02F0EE22EFCF03F0B6
:106A6000EE221200D96E3A0ED95CD8B006D0300EA4
:106A7000D95CD8A002D0D8801200D89012000900AA
:106A8000F5CFEEFFEA50E262FAD7E950E162F7D7BC
:106A90001200EE6AEA50E262FCD7E950E162F9D7EF
:0C6AA0001200EECFE6FFE82EFCD7000C41
:020000040030CA
:04000000FFFAFCFE09
:020000040000FA
:00000001FF
